:020000040800F2
:10280000304A0020012900087D6D00086B52000845
:1028100081550008693100080D7E000800000000A5
:10282000000000000000000000000000917400089B
:10283000F931000800000000856E00086576000888
:102840001B2900081B2900081B2900081B29000858
:102850001B2900081B2900081B2900081B29000848
:102860001B2900081B2900081B2900081B29000838
:102870006D3100087D3100088D3100089D31000860
:10288000AD310008BD3100081B2900081B290008D4
:102890001B2900081B2900081B2900081B29000808
:1028A0001B2900081B2900081B2900081B290008F8
:1028B0001B2900081B2900081B2900081B290008E8
:1028C0001B2900081B2900081B2900081B290008D8
:1028D0001B2900084D7D00088D7D0008CD7D000876
:1028E0001B2900081B2900081B290008DFF80CD051
:1028F00000F0B4FA0048004731AA0008304A00202E
:102900000648804706480047FEE7FEE7FEE7FEE789
:10291000FEE7FEE7FEE7FEE7FEE7FEE705770008D5
:10292000ED280008202A04DB203A00FA02F10020FA
:1029300070479140C2F1200320FA03F319439040FD
:102940007047202A04DB203A21FA02F00021704768
:1029500021FA02F3D040C2F1200291400843194607
:10296000704740EA01039B0703D009E008C9121F22
:1029700008C0042AFAD203E011F8013B00F8013B39
:10298000521EF9D27047D2B201E000F8012B491E65
:10299000FBD270470022F6E710B513460A460446FC
:1029A0001946FFF7F0FF204610BD10B5044604E0BD
:1029B0000B7800F8013B03B1491C521EF8D22046A7
:1029C00010BD421C10F8011B0029FBD1801A704772
:1029D00010B5002200E0521C835C8C5CA34201D144
:1029E000002BF8D1D8B2E1B2401A10BD30B5044680
:1029F0000020034600E05B1C934203D2E05CCD5C08
:102A0000401BF8D030BD034611F8012B00F8012B14
:102A1000002AF9D11846704730B505460020034614
:102A200000E05B1C934205D2EC5CC85C201A01D12B
:102A3000002CF6D130BD00F0004230F000400AD04A
:102A4000C10D01F56071C0F3160042EA0151C208E0
:102A500040071143704700200146704730B50B46D0
:102A6000014600202022012409E021FA02F59D42BE
:102A700005D303FA02F5491B04FA02F52844151E92
:102A8000A2F10102F1DC30BD2DE9F05F0546002026
:102A900092469B4688460646814640241BE02846CF
:102AA000414647462246FFF74CFF53465A46C01A56
:102AB000914110D3114618462246FFF733FF2D1AD5
:102AC00067EB01084F46224601200021FFF72AFF4D
:102AD00017EB00094E41201EA4F10104DFDC48463B
:102AE00031462A464346BDE8F09F2DE9FE4F804619
:102AF00081EA0300C00F0C46009021F0004123F052
:102B00000045B8EB0200A94105D240462146904657
:102B10001C460B46024623F00040104347D0270DC9
:102B2000C7F30A00C3F30A510290401A01904028EB
:102B30006BDAC3F3130040F4801B0098924620B177
:102B40000023D2EB030A63EB0B0B01985946C0F14B
:102B500040025046FFF7E6FE06460D4650465946EF
:102B6000019A00F08DF910EB08006141002487EA1A
:102B7000115284EAE7731A4340D0009A62B3019A73
:102B8000012A4FEA075215DC001B61EB02014FF0EE
:102B9000004202EA0752CDE90042001C41F58011D3
:102BA00032462B4600F08DF903B0BDE8F08F404669
:102BB0002146F9E7001B61EB0201001C41F580137F
:102BC00000185B412018A2F5001747EB030140EA0B
:102BD000D570B6196D4111E06D084FEA360645EA29
:102BE000C0754FEA0752001B61EB0201001C41F562
:102BF000801149084FEA30000019514132462B46F6
:102C000003B0BDE8F04F00F04DB90098012240003C
:102C10000023D0EB020263EBE073009821464FEAF9
:102C2000E074B8EB000061EB0401E9E783F00043D6
:102C30005BE781F0004158E72DE9FE4F81EA03048C
:102C400004F0004421F0004100944FF0000B23F009
:102C5000004350EA01045ED052EA03045BD0C3F3A0
:102C60000A54C1F30A552C44A4F2F3340194A0FB96
:102C70000254C1F3130141F48011C3F3130343F46D
:102C8000801301FB024400FB034E840A970A44EAC6
:102C9000815447EA8357A4FB076802958D0A05FB18
:102CA00007854FEA932C04FB0C542705029D4FEA3D
:102CB000065847EA1637B5EB08056EEB070C870E8A
:102CC000920E47EA811742EA8312A7FB0201B6EB94
:102CD0000B0164EB00042B0D43EA0C335E1844EB4C
:102CE0001C50DA465146E7FB0201C5F313044FEAD4
:102CF0000B3343EA14534FEA0432019C43EA0603C0
:102D0000A4F10C040294009CCDE900B400F0D9F8C1
:102D100003B0BDE8F08F00200146F9E72DE9F04D42
:102D200081EA030404F0004B21F0004514464FF003
:102D3000000A23F0004150EA050220D054EA0102C3
:102D40001DD0C5F30A570246C5F31303C1F31300A0
:102D5000C1F30A5640F4801543F48013A7EB06082C
:102D6000101BD64608F2FD3873EB050002D308F1BC
:102D7000010801E092185B41B8F1000F03DA00206E
:102D80000146BDE8F08D00204FF4801106468446D0
:102D90000EE0171B73EB050705D3121B63EB05034E
:102DA00006434CEA010C49084FEA300092185B4197
:102DB00050EA0107EDD152EA030012D082EA040082
:102DC00083EA0501084305D0101BAB4106D201225E
:102DD000002306E000224FF0004302E06FF0010202
:102DE00053101AEB06004CEB085110EB0A0041EBB4
:102DF0000B01BDE8F04D00F055B8C1F30A52C1F324
:102E0000130140F2FF3341F480119A4202DA0020AC
:102E10000146704740F233439A42A2F2334202DC49
:102E20005242FFF78EBDFFF77DBD000030B5041E96
:102E300071F1000404DB4FF00044404264EB0101F7
:102E4000141E73F1000405DB1C464FF00043524290
:102E500063EB0403994208BF904230BD064C074D16
:102E600006E0E06840F0010394E80700984710345A
:102E7000AC42F6D3FFF73EFD2CDE00084CDE000826
:102E8000202A06DBCB17203A41FA02F043EAE0732E
:102E900006E041FA02F3D040C2F12002914008431B
:102EA0001946704710B5141E73F1000408DA401C6F
:102EB00041F1000192185B411A4301D120F0010059
:102EC00010BD2DE9F04D92469B4611B1B1FA81F249
:102ED00002E0B0FA80F220329046FFF723FD04466C
:102EE0000F4640EA0A0041EA0B0153465A4608439E
:102EF00013D0114653EA010019D0C8F140025046E0
:102F0000FFF71FFD05460E46504659464246FFF75D
:102F100009FD084305D0012004E020463946BDE8FC
:102F2000F08D0020054346EAE0762C4337430A98AB
:102F30006305E40AA0EB08000022FD0A44EA4754B6
:102F40000A3002D500200146E9E701051019694160
:102F5000DDE9084500196941BDE8F04DA2E770B50B
:102F60008C1810F8015B15F0070301D110F8013B34
:102F70002A1106D110F8012B03E010F8016B01F8BB
:102F8000016B5B1EF9D12B0705D40023521E0DD413
:102F900001F8013BFAE710F8013BCB1A921C03E061
:102FA00013F8015B01F8015B521EF9D5A142D8D399
:102FB000002070BD10B51D49086880471B4948684E
:102FC00080471B49D1F8DC03804703F025FF1948EF
:102FD000816A88471848816A88471848816A884703
:102FE0001749886880471749D1F8300980470F4949
:102FF000486880471449D1F8300980471349486A26
:1030000080471349C86880471249D1F8380880477B
:103010001149086880471149486880470349486852
:1030200080470F490FA005F0ABFA10BDA80A002099
:10303000E80A0020DC090020200A0020640A0020A1
:10304000C00A002048000020E80E00205818002088
:1030500088180020081A00208C090020D40E0020B7
:103060001400002025730A0010B50A223648018892
:103070003648008803F084FE012805D132480088D4
:103080003249088004F078FB32222F48018830480A
:10309000008803F075FE012805D12B4800882C49D3
:1030A000088004F097FB642227480188294800889B
:1030B00003F066FE012805D12348008825490880D1
:1030C00004F058FBC822204801882348008803F0F8
:1030D00057FE012805D11C4800881F49088004F0CC
:1030E00069FB4FF4FA72184801881C48008803F005
:1030F00047FE012805D1144800881849088004F0CB
:103100005BFB4FF47A72104801881548008803F081
:1031100037FE012805D10C4800881149088004F0C9
:1031200033FB4FF4FA62084801880E48008803F028
:1031300027FE012805D1044800880A49088004F0C8
:103140003AFB04F0E7FA10BD2C0000203600002006
:10315000380000203A0000203C0000203E00002003
:10316000400000204200002000BFFEE710B50248EA
:1031700000F054FA10BD00005425002010B502489C
:1031800000F04CFA10BD00001025002010B50248D8
:1031900000F044FA10BD00004424002010B502489D
:1031A00000F03CFA10BD00000024002010B50248D9
:1031B00000F034FA10BD00008824002010B5024849
:1031C00000F02CFA10BD0000CC24002030B590F89F
:1031D00040500124AC40C56B6C6004686360446877
:1031E000102C04D10468A2600468E16003E0046864
:1031F000A1600468E26030BD7047704710B50446B6
:10320000204600F05BFB10BD38B532480068807B7B
:10321000401CC0B28DF800002E480068C07B401CE6
:10322000C0B28DF801002B480068007C401CC0B281
:103230008DF8020027480068407C401CC0B28DF821
:1032400003006A460C21002005F0F8F80122002155
:10325000084605F073F801221146002005F06EF8CB
:10326000052000F02BFB0321002003F09BFF132817
:1032700006D010220121002005F060F8002038BDA2
:1032800004220121002005F059F800BF002402218A
:10329000002003F087FF044624B1E2B2022100209F
:1032A00005F04CF8052000F009FB04F008000828A0
:1032B00001D10020E3E70621002003F073FFFF287F
:1032C00006D010220121002005F038F8FF20D6E7B3
:1032D000DCE700008809002038B532480068807BB0
:1032E000401CC0B28DF800002E480068C07B401C16
:1032F000C0B28DF801002B480068007C401CC0B2B1
:103300008DF8020027480068407C401CC0B28DF850
:1033100003006A460C21002005F0BCF801220021C0
:10332000084605F02BF801221146002005F026F88A
:10333000052000F0C3FA0321002003F05DFF1328ED
:1033400006D010220121002005F018F8002038BD19
:1033500004220121002005F011F800BF0024022101
:10336000002003F049FF044624B1E2B2022100200C
:1033700005F004F8052000F0A1FA04F00800082880
:1033800001D10020E3E70621002003F035FFFF28EC
:1033900006D010220121002004F0F0FFFF20D6E724
:1033A000DCE700002818002072B600BFFEE700002E
:1033B0000021074AD1610749096941F00401054A22
:1033C00011611146096941F0400111617047000027
:1033D00098250020002002400021074AD1610749BA
:1033E000096941F00201054A116111464861096904
:1033F00041F04001116170479825002000200240F3
:103400000022054BDA61054A126942F00102034BC2
:103410001A610180704700009825002000200240BA
:1034200000201E49C96801F0100139B11C49C96961
:1034300041F002011A4AD16140F010001749C968F1
:1034400001F0040139B11649C96941F00101144A7A
:10345000D16140F004001149C96901F0010169B16D
:103460000F49C96941F004010D4AD16100BF0B4900
:10347000C96921F00101094AD16100BF00BF40F2D2
:103480000111884206D10549C96921F00101034AA9
:10349000D16101E00149C86000BF704700200240CF
:1034A0009825002070B5044600F096FC054609E01A
:1034B000601C38B124B100F08FFC401BA04201D940
:1034C000032070BD1248C06800F001000028EFD151
:1034D0000F48C06800F0200020B100BF20200C4938
:1034E000C86000BF0A48C06800F0100048B908482A
:1034F000C06900F0010020B90548C06800F0040070
:1035000018B1FFF78DFF0120DBE70020D9E70000AD
:10351000002002400146002291F82100022808D034
:103520000420886300BF002081F8200000BF012034
:1035300070470868006820F00E000B681860086883
:10354000006820F001000B68186091F840300120FD
:103550009840CB6B5860012081F8210000BF00200B
:1035600081F8200000BF1046E2E7000070B5044675
:10357000002594F82100022803D00420A06301252F
:1035800048E02068006820F00E002168086020688C
:10359000006820F00100216808601F492068884207
:1035A00001D1012026E01C4914312068884201D154
:1035B00010201FE0184928312068884201D1801569
:1035C00018E015493C312068884201D1801411E08F
:1035D000114950312068884202D14FF4803009E00F
:1035E0000D4964312068884202D14FF4801001E017
:1035F0004FF08070084908394860012084F82100A4
:1036000000BF002084F8200000BF606B10B120468E
:10361000616B8847284670BD0800024070B50446BB
:10362000E06B05682068066894F840100420884024
:103630002840002846D006F00400002842D0206828
:10364000006800F0200028B92068006820F004001D
:103650002168086057492068884201D1042027E08A
:10366000544914312068884201D1402020E051495A
:1036700028312068884201D1001519E04D493C31BC
:103680002068884202D14FF4804011E0494950310E
:103690002068884202D14FF4802009E04549643116
:1036A0002068884202D14FF4800001E04FF0806032
:1036B000404908394860E06A00287AD02046E16A2B
:1036C000884776E094F84010022088402840A0B354
:1036D00006F0020088B32068006800F0200040B9BE
:1036E0002068006820F00A0021680860012084F842
:1036F000210030492068884201D1022028E02D496C
:1037000014312068884201D1202021E02949283144
:103710002068884201D140151AE026493C312068D2
:10372000884202D14FF4005012E022495031206803
:10373000884203D14FF400300AE017E01D4964319C
:103740002068884202D14FF4001001E04FF0007071
:1037500018490839486000BF002084F8200000BFE5
:10376000A06A30B32046A16A884722E094F840104E
:10377000082088402840E0B106F00800C8B1206861
:10378000006820F00E002168086094F840100120C5
:103790008840E16B48600120A06384F8210000BFED
:1037A000002084F8200000BF206B10B12046216B60
:1037B000884770BD080002400146002209B9012077
:1037C0007047164B0868C01A1423B0FBF3F0800052
:1037D000086412480838C863022081F8210008688C
:1037E000026843F6F0708243D1E901031843CB68C5
:1037F00018430B6918434B6918438B691843CB690D
:10380000184302430868026000208863012081F8A1
:103810002100002081F8200000BFD1E7080002400D
:103820002DE9F04104460D4616461F464FF00008AC
:1038300000BF94F82000012802D10220BDE8F081E9
:10384000012084F8200000BF94F8210001282CD129
:10385000022084F821000020A0632068006820F086
:103860000100216808603B46324629462046FFF7A2
:10387000ADFCE06A30B12068006840F00E002168BD
:1038800008600BE02068006820F0040021680860F0
:103890002068006840F00A0021680860206800681D
:1038A00040F001002168086006E000BF002084F8B5
:1038B000200000BF4FF002084046BFE770B5044645
:1038C00000F08AFA06462546681C10B104480078C4
:1038D000054400BF00F080FA801BA842FAD370BDF7
:1038E000080000202DE9F04104460E46012700257E
:1038F00000BF2648007E012802D10220BDE8F081E9
:1039000001202249087600BF2068022813D14CF21A
:103910005030FFF7C7FD90BB0120FFF749FD4CF287
:103920005030FFF7BFFD07461948006920F004003A
:103930001749086123E04CF25030FFF7B3FDF0B9AE
:103940004FF0FF303060A56812E02846FFF744FDD5
:103950004CF25030FFF7A6FD07460D48006920F0F5
:1039600002000B4908610FB1356007E005F580657D
:10397000D4E9021001EB8020A842E6D800BF00BFC6
:1039800000200249087600BF3846B7E79825002096
:10399000002002400348006940F0800001490861AE
:1039A00000207047002002402DE9FE4F05468B465F
:1039B00017469846012600240020029000BF2448A4
:1039C000007E012802D10220BDE8FE8F012020499F
:1039D000087600BF4CF25030FFF764FD064686BB08
:1039E000012D02D10120029006E0022D02D1022019
:1039F000029001E00420029000241EE02201B9465A
:103A0000C24648465146FEF79CFF80B20190022014
:103A100000FB04B000900199FFF7F2FC4CF250302B
:103A2000FFF740FD06460B48006920F001000949F8
:103A3000086106B104E0601CC4B202988442DDDB78
:103A400000BF00BF00200249087600BF3046BBE738
:103A5000982500200020024000200849096901F053
:103A6000800151B10649054A51600649516011462D
:103A7000096901F0800101B1012070470020024076
:103A800023016745AB89EFCD2DE9F84703460022B6
:103A900094466EE14FF0010808FA02F4D1F8008074
:103AA00008EA0400A0427DD1DFF8DCA2D1F804804E
:103AB000A8EB0A09D0453AD014DCB8F1030F50D076
:103AC00009DCB8F1000F31D0B8F1010F1CD0B8F10A
:103AD000020F49D120E0B8F1110F18D0B8F1120F40
:103AE00042D11EE0B9F5881F25D006DCB9F5803F2C
:103AF00020D0B9F5801F37D11AE0B9F5001F18D0D2
:103B0000B9F5041F30D117E0D1F80CC02DE0D1F881
:103B10000C8008F1040C28E0D1F80C8008F1080CA6
:103B200023E0D1F80C8008F10C0C1EE000BF00BFB0
:103B300000BF00BF00BF00BFD1F80880B8F1000F80
:103B400002D14FF0040C0BE0D1F80880B8F1010F5E
:103B500003D14FF0080C1C6102E04FF0080C5C61CF
:103B600003E04FF0000C00E000BF00BFFF2801D8C9
:103B7000984601E003F104084646FF2802D84FEAC0
:103B8000820803E0A2F108084FEA88084746D6F801
:103B900000804FF00F0909FA07F928EA09080CFA22
:103BA00007F900E088E048EA0908C6F80080D1F883
:103BB000048008F08058B8F1805F7DD100BFDFF845
:103BC000CC81D8F8188048F00108DFF8C091C9F816
:103BD0001880C846D8F8188008F00108CDF8008091
:103BE00000BF00BF4FEAB9384FEA920958F8295090
:103BF0004FEA82784FEA18794FF00F0808FA09F86F
:103C000025EA0805DFF88881434502D14FF0000816
:103C100016E0DFF88081434502D14FF001080FE044
:103C2000DFF87481434502D14FF0020808E0DFF865
:103C30006C81434502D14FF0030801E04FF00408C6
:103C40004FEA82794FEA197908FA09F848EA050536
:103C5000DFF84C814FEA920948F82950D1F80480E6
:103C600008F48018B8F5801F0AD1DFF83881D8F839
:103C7000008048EA0008DFF82C91C9F8008009E0CC
:103C8000DFF82081D8F8008028EA0008DFF81491D6
:103C9000C9F80080D1F8048008F40018B8F5001FB6
:103CA00010D1DFF8008108F10408D8F8008048EA54
:103CB0000008DFF8F09000E05AE009F10409C9F8C3
:103CC00000800DE0DFF8DC8008F10408D8F80080FF
:103CD00028EA0008DFF8CC9009F10409C9F800804F
:103CE000D1F8048008F40038B8F5003F0ED1DFF8B1
:103CF000B480A8F10408D8F8008048EA0008DFF88A
:103D0000A490A9F10409C9F800800DE0DFF89480BF
:103D1000A8F10408D8F8008028EA0008DFF88490A9
:103D2000A9F10409C9F80080D1F8048008F48038AA
:103D3000B8F5803F0ED1DFF86C80A8F10808D8F8FC
:103D4000008048EA0008DFF85C90A9F10809C9F88A
:103D500000800DE0DFF84C80A8F10808D8F800805A
:103D600028EA0008DFF83C90A9F10809C9F80080AA
:103D7000521CD1F8008028FA02F8B8F1000F7FF445
:103D800089AEBDE8F8870000000011100010024065
:103D900000080140000C01400010014000140140E7
:103DA0000800014008040140024693680B400BB133
:103DB000012000E00020704710B5C26821EA02032C
:103DC00002EA010443EA0443036110BD0AB1016140
:103DD00001E00B0403617047014800687047000070
:103DE0000000002070B504460CB9012070BD4CF6EF
:103DF000CC402168086045F2555021680860D4E93C
:103E0000001048602168A0688860FFF7E5FF05465C
:103E10000DE0FFF7E1FF401B41F23C31884206D93B
:103E20002068C06800F0030008B10320DEE72068C6
:103E3000C06800F003000028EBD14AF6AA202168F0
:103E400008600020D2E701464AF6AA200A681060FE
:103E50000020704703480068034909780844014975
:103E600008607047000000200800002010B50848D6
:103E7000006840F0100006490860032000F0A8F830
:103E80000F2000F007F800F02BF8002010BD000014
:103E90000020024070B504460E4800784FF47A7155
:103EA000B1FBF0F00C490968B1FBF0F5284600F0D1
:103EB000D6FD08B1012070BD102C07D2002221468A
:103EC000501E00F047F80548046001E00120F2E7C9
:103ED0000020F0E7080000200C0000200400002073
:103EE00008B500BF1148806940F001000F498861A2
:103EF0000846806900F00100009000BF00BF00BFCD
:103F00000846C06940F08050C8610846C06900F0AA
:103F10008050009000BF00BF00BF0549486820F0F6
:103F2000E06040F00070486000BF08BD0010024033
:103F30000000014001460846002809DB00F01F038D
:103F400001229A4043099B0003F1E023C3F80021BA
:103F500000BF70472DE9F05F80460D4616460027EA
:103F600004F04AFB074639462A46334601F007006B
:103F7000C0F1070ABAF1040F02D94FF0040A01E0B8
:103F8000C0F1070AD14600F1040ABAF1070F02D2C4
:103F90004FF0000A01E0A0F1030AD4464FF0010AF5
:103FA0000AFA09FAAAF1010A0AEA020A0AFA0CFA5A
:103FB0004FF0010B0BFA0CFBABF1010B0BEA030BFF
:103FC0004AEA0B042146404604F01EFBBDE8F09F80
:103FD00000BF00F00702064B19684FF6FF031940B7
:103FE000044B0B4343EA0221014B196000BF7047A9
:103FF0000CED00E00000FA0500BF00BF00BF00BFED
:1040000000BFBFF34F8F00BF00BF00BF094800686B
:1040100000F4E06008490843001D0649086000BF3D
:1040200000BF00BFBFF34F8F00BF00BF00BF00BF86
:1040300000BFFDE70CED00E00000FA0570B5044696
:104040000D460CB9012070BD5A48006800F0070009
:10405000A8420ED25748006820F00700284355496F
:1040600008600846006800F00700A84201D001205F
:10407000E9E7207800F0020002281DD1207800F046
:104080000400042805D14C48406840F4E0604A49E7
:104090004860207800F00800082805D146484068AC
:1040A00040F46050444948604348406820F0F000C4
:1040B000A168084340494860207800F0010078B3C7
:1040C0006068012806D13C48006800F4003090B9CF
:1040D0000120B8E76068022806D13748006800F080
:1040E000007040B90120AEE73348006800F00200DC
:1040F00008B90120A7E73048406820F00300616854
:1041000008432D494860FFF767FE064609E0FFF7C0
:1041100063FE801B41F28831884202D9032092E776
:1041200007E02548406800F00C006168B0EB810FA3
:10413000EDD12048006800F00700A8420ED91D48C4
:10414000006820F0070028431A4908600846006804
:1041500000F00700A84201D0012074E7207800F0A9
:104160000400042807D11448406820F4E060E168A6
:10417000084311494860207800F00800082808D159
:104180000D48406820F46050216940EAC1000A49A6
:10419000486000F03FF808494968C1F30311074A35
:1041A000515CC8400649086006480068FFF772FE87
:1041B000002048E70020024000100240F2D400082E
:1041C0000C00002004000020014800687047000037
:1041D0000C00002000B5FFF7F7FF04494968C1F360
:1041E0000221034A515CC84000BD0000001002409B
:1041F00002D5000800B5FFF7E7FF04494968C1F39D
:10420000C221034A515CC84000BD000000100240BA
:1042100002D5000870B500210022002400230020F0
:10422000134D696801F00C05F5B1042D02D0082D7D
:1042300019D101E00F4819E00F4DC1F38346AB5D82
:1042400001F4803555B10A4D6D68C5F340450B4EFC
:10425000725D084D5D43B5FBF2F402E0084D03FBCF
:1042600005F4204602E000BF024800BF00BF70BD59
:104270000010024000127A00E0D40008F0D40008D8
:1042800000093D00F8B504460CB90120F8BD2078BE
:1042900000F00100002878D0F848406800F00C00D9
:1042A00004280CD0F548406800F00C00082811D113
:1042B000F248406800F48030B0F5803F0AD1EF4802
:1042C000006800F4003000285FD0606800285CD1EE
:1042D0000120DBE700BF6068B0F5803F06D1E7480A
:1042E000006840F48030E549086028E0606858B90B
:1042F000E248006820F48030E04908600846006821
:1043000020F4802008601AE06068B0F5A02F0BD17F
:10431000DA48006840F48020D84908600846006800
:1043200040F4803008600AE0D448006820F480300F
:10433000D24908600846006820F48020086000BF69
:10434000606888B1FFF748FD054606E0FFF744FDC9
:10435000401B642801D9032098E7C848006800F48E
:1043600000300028F2D010E0FFF736FD054606E0E9
:10437000FFF732FD401B642801D9032086E7BF48C0
:10438000006800F400300028F2D1207800F002002C
:10439000022857D1B948406800F00C0050B1B74826
:1043A000406800F00C00082818D1B448406800F4B8
:1043B000803098B9B148006800F0020020B120694F
:1043C000012801D0012061E7AC48006820F0F80026
:1043D000616940EAC100A949086033E02069E8B199
:1043E0000120A7490860FFF7F7FC054606E0FFF744
:1043F000F3FC401B022801D9032047E79F480068CF
:1044000000F002000028F2D09C48006820F0F8007C
:10441000616940EAC1009949086013E000209849A9
:104420000860FFF7D9FC054606E0FFF7D5FC401B06
:10443000022801D9032029E79048006800F0020013
:104440000028F2D1207800F0080008282DD1A069BA
:10445000B8B101208B490860FFF7BEFC054606E0B5
:10446000FFF7BAFC401B022801D903200EE783485E
:10447000406A00F002000028F2D0012002F004FDA2
:1044800013E000207F490860FFF7A6FC054606E020
:10449000FFF7A2FC401B022801D90320F6E677486B
:1044A000406A00F002000028F2D1207800F00400F9
:1044B000042873D100277148C06900F0805070B99A
:1044C00000BF6E48C06940F080506C49C861084622
:1044D000C06900F08050009000BF00BF01276A480B
:1044E000006800F48070B0B96748006840F48070DC
:1044F00065490860FFF770FC054606E0FFF76CFCB5
:10450000401B642801D90320C0E65F48006800F41E
:1045100080700028F2D000BFE068012806D157481B
:10452000006A40F001005549086227E0E06858B988
:104530005248006A20F00100504908620846006AAB
:1045400020F00400086219E0E06805280BD14B4810
:10455000006A40F00400494908620846006A40F0D9
:10456000010008620AE04548006A20F00100434962
:1045700008620846006A20F00400086200BFE06894
:10458000A0B1FFF729FC054609E0FFF725FC401B19
:1045900041F28831884202D9032077E622E0374889
:1045A000006A00F002000028EFD012E0FFF714FCD0
:1045B000054608E0FFF710FC401B41F288318842B5
:1045C00001D9032062E62D48006A00F002000028AD
:1045D000F0D1012F05D12948C06920F0805027492A
:1045E000C86100BFE069C8B32448406800F00C000F
:1045F000082860D0E069022848D1002020490866D8
:10460000FFF7EAFB054606E0FFF7E6FB401B022842
:1046100001D903203AE61948006800F0007000282C
:10462000F2D1206AB0F5803F07D11448406820F4E9
:104630000030A168084311494860D4E908010843E3
:104640000E49496821F4741108430C49486001205F
:104650000B490866FFF7C0FB054607E03DE0FFF7A2
:10466000BBFB401B022801D903200FE6034800686A
:1046700000F000700028F2D02FE00000001002408F
:104680000000424280044242007000400020144971
:104690000866FFF7A1FB054606E0FFF79DFB401B00
:1046A000022801D90320F1E50E48006800F00070EF
:1046B0000028F2D111E0E069012800D1E6E50948BF
:1046C000466806F48031206A814204D106F47011F4
:1046D000606A814201D00120D8E50020D6E50000C3
:1046E000000042420010024010B504460CB90120FF
:1046F00010BD606A38B96068B0F5827F00D105E00E
:104700000021E16102E00021216161610021A162DB
:1047100094F8510028B9002084F85000204600F099
:1047200043F8022084F851002068006820F040001F
:1047300021680860A08800F48270218901F4044196
:104740000843A18901F400610843217C01F00201C2
:104750000843217D01F001010843218B01F4007120
:104760000843217F01F0380108432021095D01F051
:1047700080010843218D01F400510843216808603D
:104780000421A06901EA1040216848602068C069DE
:1047900020F400602168C86100206065012084F871
:1047A00051000020A4E7000010B586B004460020A8
:1047B00002900390049005903449206888422ED1DD
:1047C00000BF3348806940F4805031498861084611
:1047D000806900F48050019000BF00BF00BF084610
:1047E000806940F0040088610846806900F0040098
:1047F000019000BF00BFA020029002200390032080
:10480000059002A92348FFF73FF9402002900020BD
:104810000390049002A91F48FFF736F933E01E49C0
:10482000206888422FD100BF1948C06940F48040F9
:104830001749C8610846C06900F48040019000BF74
:1048400000BF00BF0846806940F008008861084644
:10485000806900F00800019000BF00BF4FF42040C5
:104860000290022003900320059002A90B48FFF755
:104870000BF94FF48040029000200390049002A9AD
:104880000648FFF701F906B010BD000000300140F6
:10489000001002400008014000380040000C0140B8
:1048A0002DE9F84304460F4616461D46FFF794FAD5
:1048B0008046B14694F85100012802D00220BDE89C
:1048C000F88307B10EB90120F9E700BF94F8500052
:1048D000012801D10220F2E7012084F8500000BF36
:1048E000032084F85100002060652763A686E686D1
:1048F000A063A087E08760642064A068B0F5004FE3
:104900000BD12068006820F0400021680860206812
:10491000006840F48040216808602068006800F06A
:104920004000402805D02068006840F04000216821
:104930000860E068B0F5006F37D1606810B1B9F178
:10494000010F09D1206B00882168C860206B801C92
:104950002063E08E401EE08623E02068806800F03F
:10496000020002280AD1206B00882168C860206BF1
:10497000801C2063E08E401EE08612E0FFF72CFAD8
:10498000A0EB0800A84201D3681C00B94DB9012072
:1049900084F8510000BF002084F8500000BF0320BD
:1049A0008DE7E08E0028D8D136E0606810B1B9F10B
:1049B000010F09D1206B007821680873206B401C1F
:1049C0002063E08E401EE08623E02068806800F0CF
:1049D000020002280AD1206B007821680873206B3E
:1049E000401C2063E08E401EE08612E0FFF7F4F9E1
:1049F000A0EB0800A84201D3681C00B94DB9012002
:104A000084F8510000BF002084F8500000BF03204C
:104A100055E7E08E0028D8D142462946204602F0CC
:104A2000A8FC08B120206065A06850B900BF002034
:104A300000902068C068009020688068009000BFE7
:104A400000BF012084F8510000BF002084F850000E
:104A500000BF606D08B1012031E700202FE770B57D
:104A600004462546681EB0F1807F01D301200FE087
:104A7000681E4FF0E02148610F214FF0FF3003F036
:104A8000C3FD00204FF0E02188610720086100206D
:104A900070BD704770B50446002520684069C0F3BA
:104AA000C01594F84100212817D1B5B100BF00BF4F
:104AB0002168143151E8001F21F080002168143171
:104AC00041E80002002AF3D100BFA06B10B1A06B37
:104AD000FEF720FD204602F095FF20684069C0F3F4
:104AE000801594F84200222817D1B5B100BF00BF4D
:104AF0002168143151E8001F21F040002168143171
:104B000041E80002002AF3D100BFE06B10B1E06B76
:104B1000FEF700FD204602F02FFF002070BD704719
:104B20002DE9F84F0446206805682068C6682068AB
:104B300047694FF00009CA4605F00F09B9F1000FA7
:104B40000AD105F0200038B106F0200020B120463F
:104B500002F06BFFBDE8F88FB9F1000F7BD007F0D2
:104B6000010018B906F49070002874D005F0010017
:104B700030B106F4807018B1606C40F001006064E0
:104B800005F0040030B107F0010018B1606C40F08E
:104B90000200606405F0020030B107F0010018B1B6
:104BA000606C40F00400606405F0080048B106F055
:104BB000200010B907F0010018B1606C40F0080047
:104BC0006064606C002845D005F0200028B106F034
:104BD000200010B1204602F028FF20684069C0F391
:104BE000801A606C00F0080010B9BAF1000F2CD0E8
:104BF000204602F0C1FE2068406900F0400000B38A
:104C000000BF00BF2168143151E8001F21F04000AF
:104C10002168143141E80002002AF3D100BFE06BA3
:104C200050B17748E16B4863E06BFEF79FFC88B1B9
:104C3000E06B416B88470DE02046FFF770FF09E00D
:104C400009E02046FFF76BFF04E02046FFF767FF0F
:104C5000002060647EE7206B012877D105F010000A
:104C6000002873D006F010000028FAD000BF002002
:104C7000009020680068009020684068009000BFA5
:104C800000BF2068406900F0400000285FD0E06B62
:104C9000006840681FFA80F8B8F1000F55D0A08D69
:104CA000404552DDA4F82E80E06B8069202843D077
:104CB00000BF00BF21680C3151E8001F21F4807053
:104CC00021680C3141E80002002AF3D100BF00BF87
:104CD00000BF2168143151E8001F21F00100216854
:104CE000143141E80002002AF3D100BF00BF00BF29
:104CF0002168143151E8001F21F04000216814316F
:104D000041E80002002AF3D100BF202084F84200CD
:104D10000020206300BF00BF21680C3151E8001F54
:104D200021F0100021680C3141E80002002AF3D183
:104D300000BFE06BFEF7EEFB02206063A08DE28D0A
:104D4000801A81B22046FFF7A4FE03E742E0A08D5F
:104D5000E18D401A1FFA80F8E08DD0B3B8F1000F52
:104D600037D000BF00BF21680C3151E8001F21F48B
:104D7000907021680C3141E80002002AF3D100BF95
:104D800000BF00BF2168143151E8001F21F001006D
:104D90002168143141E80002002AF3D100BF20202D
:104DA00084F842000020206300BF00BF21680C315E
:104DB00051E8001F21F0100021680C3141E8000289
:104DC000002AF3D100BF0220606341462046FFF76E
:104DD00060FEBFE605F0800030B106F0800018B13B
:104DE000204602F083FFB5E605F0400030B106F042
:104DF000400018B1204602F0F5FDABE600BFA9E681
:104E0000D777000810B504460CB9012010BDA06981
:104E100000B100E000BF94F8410028B9002084F8F8
:104E20004000204600F02AF8242084F84100206841
:104E3000C06820F400502168C860204602F074FE6B
:104E40002068006920F4904021680861206840696A
:104E500020F02A00216848612068C06840F40050B2
:104E60002168C86000206064202084F8410084F834
:104E700042000020606300BFC8E7000010B586B0A4
:104E8000044600200290039004900590A7492068F2
:104E900088426AD100BFA648806940F48040A44996
:104EA00088610846806900F48040019000BF00BF1F
:104EB00000BF0846806940F00400886108468069A8
:104EC00000F00400019000BF00BF481502900220CE
:104ED00003900320059002A99648FEF7D5FD4FF4F4
:104EE0008060029000200390049002A99148FEF790
:104EF000CBFD9148914908600020486000218F480F
:104F000081608021C1600021016141618161C161D5
:104F1000FEF752FC08B1FEF747FA00BF8748E0638E
:104F2000446200BF844814388549086010204860F6
:104F30000021834881608021C160002101614161BD
:104F40008161C161FEF738FC08B1FEF72DFA00BFA0
:104F50007B48A063446200BF002211462520FEF773
:104F6000F9FF2520FEF7E6FFDDE07649206888425C
:104F70006AD100BF6E48C06940F400306C49C86116
:104F80000846C06900F40030019000BF00BF00BFB8
:104F90000846806940F0040088610846806900F096
:104FA0000400019000BF00BF042002900220039083
:104FB0000320059002A95F48FEF766FD08200290D5
:104FC00000200390049002A95A48FEF75DFD5A485C
:104FD00014305D4908600020486000215A48816013
:104FE0008021C1600021016141618161C161FEF7E1
:104FF000E3FB08B1FEF7D8F900BF5348E063446211
:1050000000BF4D48283051490860102048600021F9
:105010004E4881608021C160002101614161816150
:10502000C161FEF7C9FB08B1FEF7BEF900BF4748F2
:10503000A063446200BF002211462620FEF78AFFCB
:105040002620FEF777FF6EE04149206888426AD14A
:1050500000BF3748C06940F480203549C861084620
:10506000C06900F48020019000BF00BF00BF084667
:10507000806940F0080088610846806900F00800F7
:10508000019000BF00BF081502900220039003208A
:10509000059002A92F48FEF7F7FC4FF4006002903C
:1050A00000200390049002A92A48FEF7EDFC224854
:1050B000283829490860002048600021264881607E
:1050C0008021C1600021016141618161C161FEF700
:1050D00073FB08B1FEF768F900BF1F48E063446244
:1050E00000BF15483C381D49086010204860002169
:1050F0001A4881608021C1600021016141618161A4
:10510000C161FEF759FB08B1FEF74EF900BF134825
:10511000A063446200BF002211462720FEF71AFF59
:105120002720FEF707FF06B010BD00000038014041
:1051300000100240000801405800024000240020F6
:10514000442400200044004088240020CC24002077
:1051500000480040000C014010250020542500208C
:1051600070B504460D46164694F8420020280BD12F
:1051700005B10EB9012070BD0020206332462946DA
:10518000204602F04FFDF6E70220F4E77047704733
:10519000F7B50446154694F84100202836D1019809
:1051A00000B10DB90120FEBD01982062A584E584FF
:1051B00000206064212084F841001548A16B8862BA
:1051C0001448A16BC8621448A16B08630020A16B4E
:1051D000486301AE23681A1D31682B46A06BFEF7A9
:1051E0001FFB6FF040002168086000BF00BF21680E
:1051F000143151E8001F41F080002168143141E86A
:105200000002002AF3D100BF0020CCE70220CAE749
:10521000137900086B790008EB77000810B5044695
:105220000B492068884203D10A48016B88470EE089
:1052300009492068884203D10848016B884706E085
:1052400007492068884202D10648016B884710BD93
:1052500000380140DC09002000440040200A002002
:1052600000480040640A0020704700BFFEE7014686
:105270000A2291FBF2F302FB13120A2391FBF3F3D0
:1052800002EB0312D0B2704708B500BF1E48406958
:1052900040F001001C4948610846406900F00100E7
:1052A000009000BF00BF002211460C20FEF752FE06
:1052B0000C20FEF73FFE002211460D20FEF74AFEAD
:1052C0000D20FEF737FE002211460E20FEF742FEAB
:1052D0000E20FEF72FFE002211460F20FEF73AFEA9
:1052E0000F20FEF727FE002211461020FEF732FEA7
:1052F0001020FEF71FFE002211461120FEF72AFEA5
:105300001120FEF717FE08BD0010024000B585B061
:105310000020019002900390049000BF3E488069F5
:1053200040F010003C4988610846806900F0100098
:10533000009000BF00BF00BF0846806940F0200019
:1053400088610846806900F02000009000BF00BF1F
:1053500000BF0846806940F0040088610846806903
:1053600000F00400009000BF00BF00BF0846806945
:1053700040F0080088610846806900F0080000904D
:1053800000BF00BF01224FF4C0412448FEF71EFDBC
:10539000002241F612012248FEF718FD012241F2D7
:1053A00003012048FEF712FD0022E0211D48FEF710
:1053B0000DFD4FF4C04001900120029000200390A9
:1053C0000220049001A91548FEF75EFB41F6120089
:1053D000019001200290002003900220049001A976
:1053E0000F48FEF751FB41F2E300019001200290CB
:1053F000002003900320049001A90A48FEF744FB13
:105400004FF40070019000200290039001A905481C
:10541000FEF73AFB05B000BD00100240001001404D
:1054200000080140000C014010B50748074908601A
:10543000062048604FF4EA7104488160FEF7D2FC10
:1054400008B1FDF7B1FF10BD003000406C22002014
:1054500010B50E480E4908604FF482704860002174
:105460000B488160C160016141614FF4007181614D
:105470000821C16100210162416281620A21C16289
:10548000FFF732F908B1FDF78FFF10BD0030014082
:105490007822002010B50E480E4908604FF4827043
:1054A000486000210B488160C160016141614FF497
:1054B000007181610021C1610162416281620A2142
:1054C000C162FFF711F908B1FDF76EFF10BD0000D2
:1054D00000380040D022002010B50B480B4908606E
:1054E0004FF416504860002108488160C160016196
:1054F0000C21416100218161C161FFF783FC08B18A
:10550000FDF752FF10BD00000038014028230020A5
:1055100010B50B480B4908604FF416504860002145
:1055200008488160C16001610C21416100218161F5
:10553000C161FFF767FC08B1FDF736FF10BD000041
:10554000004400407023002010B50B480B49086050
:105550004FF416504860002108488160C160016125
:105560000C21416100218161C161FFF74BFC08B151
:10557000FDF71AFF10BD000000480040B8230020CE
:1055800000BFFEE72DE9F04104460D46164614B96A
:105590000020BDE8F081082E01DA0020F9E7B01EF6
:1055A00081B2284601F0CCFB0746A81910F8018CFF
:1055B0004FF6FF7000EA0828A81910F8020C40EA1C
:1055C0000808B84501D00020E3E728782070687803
:1055D0006070A878000260806088E9780843608085
:1055E0006078062802D1281DA06013E0607810289A
:1055F00009D128790002A080A08869790843A08099
:10560000E81DA06006E028790002A080A0886979E2
:105610000843A0800120BCE770B50546AB2D03D040
:1056200003DCAB2D02D202E078E35BE1DBE1A90011
:10563000794449688F440000C6030000C803000095
:10564000CA030000CC030000CE030000D00300001A
:10565000D2030000D4030000D6030000D8030000EA
:10566000DA030000DC030000EC030000EE0300009E
:10567000F0030000F2030000F4030000F603000052
:10568000F8030000FA030000FC030000FE03000022
:10569000F2040000F4040000F6040000F804000026
:1056A00002050000100500001205000014050000AE
:1056B0001605000022050000280500002A0500004C
:1056C0002C0500002E0500003A05000046050000EC
:1056D0004C05000052050000580500005E05000062
:1056E0006405000066050000680500006A0500000A
:1056F0007405000082050000840500008605000096
:10570000880500009405000096050000980500003B
:105710009A050000A6050000A8050000AA050000E3
:10572000AC050000B8050000C6050000C805000073
:10573000CA050000CC050000CE050000D005000021
:10574000DC050000DE050000E0050000E2050000C9
:10575000E4050000E60500004609000046090000D7
:1057600046090000460900004609000046090000FD
:1057700046090000460900004609000046090000ED
:1057800046090000460900004609000046090000DD
:1057900046090000460900004609000046090000CD
:1057A00046090000460900004609000046090000BD
:1057B00046090000460900004609000046090000AD
:1057C0004609000046090000F2050000F40500004B
:1057D000F6050000F8050000FA050000FC050000D1
:1057E000FE0500000006000002060000040600009E
:1057F00006060000080600001E0600002006000045
:1058000022060000240600002606000028060000EC
:105810002A0600002C0600002E06000030060000BC
:1058200032060000340600004A0600004C06000064
:105830004E0600005006000052060000540600000C
:1058400056060000580600005A0600005C060000DC
:105850005E06000060060000760600007806000084
:105860007A0600007C0600007E060000800600002C
:1058700082060000840600008606000088060000FC
:105880008A0600008C060000A2060000A4060000A4
:10589000A6060000A8060000AA060000AC0600004C
:1058A000AE060000B0060000B2060000B40600001C
:1058B000B6060000B8060000CE060000D0060000C4
:1058C000D2060000D4060000D6060000D80600006C
:1058D000DA060000DC060000DE060000E00600003C
:1058E000E2060000F32D7DD029DCA5F1AC004728AD
:1058F00079D2DFE800F0F6F5F4F3F2F1F0EFEEED37
:10590000ECEBEAE9E8E7E6E5E4E3E2E1E0DFDEDD4F
:10591000DCDBDAD9D8D7D6D5D4D3D2D1D0CFCECD3F
:10592000CCCBCAC9C8C7C6C5C4C3C2C1C0BFBEBD2F
:10593000BCBBBAB9B8B7B6B5B4B3B2B1B00040F2F7
:105940001711681A8D427CD017DCA5F1F4002328CA
:10595000CED2DFE800F0E9E8E7E6E5E4E3E2E1E003
:10596000DFDEDDDCDBDAD9D8D7D6D5D4D3D2D1D0BF
:10597000CFCECDCCCBCAC9C8C700122862D015DCA7
:105980001228B5D2DFE810F02F00A202A602AA0268
:10599000AB02AC02AD02AE02AF02B002B102B20283
:1059A000B302B402BB02BC02BD02BE021B284AD035
:1059B0000DDCA0F1130008289AD2DFE810F0A50250
:1059C000AC02AD02AE02AF02B002B102B8022028B2
:1059D0003AD00BDC1C2838D01D2837D01E2836D0F2
:1059E0001F2801E02FE233E032D1B4E2212830D089
:1059F00022282FD0A0F2D1200028F5D1BBE200BF91
:105A000000BF00BF00BF00BF00BF00BF00BF00BF9E
:105A100000BF00BFF94800EB45067078317840EAD6
:105A20000124AEE200BF00BF00BF00BF00BF00BF47
:105A300000BF00BF00BFA5F10C00F14931F81040D4
:105A40009FE23FE25FE276E286E278E27BE27BE29F
:105A500095E288E288E2F5E1F3E1F1E1EFE1EDE1E1
:105A6000EBE1E9E1E7E1E5E1DEE1DCE1DAE1D8E122
:105A7000D6E1D4E1D2E1BBE1B9E1B7E1B5E1B3E10F
:105A8000B1E1AFE1A9E1A3E19DE198E190E18EE10F
:105A90008CE18AE188E186E184E182E180E17EE1D6
:105AA0007CE17AE178E176E174E172E170E16EE146
:105AB0006CE16AE15EE15CE15AE158E156E154E1F2
:105AC00052E150E14EE14CE14AE148E13CE13AE18A
:105AD00038E136E134E132E130E12EE12CE12AE136
:105AE00028E126E1EAE1E2E1E0E1DEE1DCE1DAE120
:105AF000D8E1D6E1D4E1D2E1D0E1CEE1CCE1CAE116
:105B0000C8E1C6E1C4E1C2E1C0E1BEE1B6E1B4E191
:105B1000B2E1B0E1AEE1A6E1A4E1A2E1A0E19EE143
:105B20009CE19AE198E196E18EE100BF00BF00BFE1
:105B3000A5F11600B3490C5C23E2B2480E38817D12
:105B4000407D41EA00241CE200BF00BF00BFA5F178
:105B50001B00AC490A390C5C13E2AB48048C10E220
:105B600000BF00BF00BFA5F12000A6490E390C5CA4
:105B700007E2A648008800F5FA6084B201E2A34873
:105B80008478FEE1A148C478FBE1A0480479F8E1FB
:105B90009E484479F5E19D488479F2E100BF00BF59
:105BA00000BFA5F12A009A490C5CEAE198480E383A
:105BB000817D407D41EA0024E3E100BF00BF00BFDA
:105BC000A5F12F0092490A390C5CDAE100BF00BF51
:105BD00000BFA5F133008E490E390C5CD1E100BF46
:105BE00000BF00BFA5F1370189480930445CC8E116
:105BF00087480E38017FC07E41EA0024C1E100BF22
:105C000000BF00BF00BF00BFA5F13C007D49891F58
:105C10000C5CB6E100BF00BF00BF00BF00BFA5F134
:105C200042007B49891F0C5CABE100BF00BF00BF95
:105C300000BF00BF00BF00BF00BF00BF00BF00BF6C
:105C4000A5F164016E486A3030F81140204603F037
:105C500068F9044695E100BF00BF00BF00BF00BF68
:105C600000BF00BF00BF00BF00BF00BFA5F17001B3
:105C70006348523030F81140204603F052F9044690
:105C80007FE100BF00BF00BF00BF00BF00BF00BF7B
:105C900000BF00BF00BF00BFA5F17C015848E23043
:105CA00030F81140204603F03CF9044669E100BF9A
:105CB00000BF00BF00BF00BF00BF00BF00BF00BFEC
:105CC00000BF00BFA5F188014D483A3030F81140BF
:105CD000204603F026F9044653E100BF00BF00BF91
:105CE00000BF00BF00BF00BF00BF00BF00BF00BFBC
:105CF000A5F194014248CA3030F81140204603F023
:105D000010F904463DE100BF00BF00BF00BF00BF67
:105D100000BF00BF00BF00BF00BF00BFA5F1A001D2
:105D20003748B23030F81140204603F0FAF8044604
:105D300027E100BF00BF00BF00BF00BF00BF00BF22
:105D400000BF00BF00BF00BFA5F1AC012C488230EE
:105D500030F81140204603F0E4F8044611E100BF9A
:105D600000BF00BF00BF00BF00BF00BF00BF00BF3B
:105D700000BF00BFA5F1B80121489A3030F81140AA
:105D8000204603F0CEF80446FBE000BF00BF00BF92
:105D900000BF00BF00BF00BF00BF00BF00BF00BF0B
:105DA00000BF00BF00BF00BF00BF00BF00BF00BFFB
:105DB000A5F1C4011248FA3030F81140E1E015486D
:105DC000B0F80E43DDE01348B0F8100384B2D8E019
:105DD0001048B0F8140384B2D3E00E48B0F81803AA
:105DE00084B2CEE000BF00BF00BF00BF00BF00BF55
:105DF000A5F1DC01084830F81140C2E01400002091
:105E0000D40C00205600002058180020C00A0020A2
:105E1000F60E0020E80A0020040E002000BF00BF9C
:105E200000BF00BF00BF00BFA5F1E301564830F836
:105E30001140A6E000BF00BF00BF00BF00BF00BF11
:105E400000BF00BF00BF00BFA5F1EA014E480E3001
:105E500030F8114095E000BF00BF00BF00BF00BF99
:105E600000BF00BF00BFA5F1F5014748243030F85E
:105E7000114086E000BF00BF00BF00BFA5F1FE01DA
:105E80004148363030F811407BE000BF00BF00BF12
:105E900000BF00BF00BF00BF00BF00BF00BF00BF0A
:105EA00000BF00BF00BF00BF00BF00BF00BFA5F222
:105EB00003113548403030F8114062E03348B0F803
:105EC00090435EE03148B0F892435AE02F48B0F872
:105ED000944356E02D48B0F8964352E000BF00BF0F
:105EE00000BF00BF00BF00BF00BF00BF00BF00BFBA
:105EF000A5F58D7124486E3030F8114041E000BFA7
:105F000000BF00BF00BF00BFA5F225111E488430AE
:105F100030F8114035E000BF00BF00BF00BF00BF38
:105F2000A5F22B111848903030F8114029E017489D
:105F3000B0F8C64325E01548B0F8C84321E013483F
:105F4000B0F8CA431DE000BFA5F59A710E48A23013
:105F500030F8114015E000BFA5F59B710A48A63046
:105F600030F811400DE000BFA5F59C710648AA303D
:105F700030F8114005E0054890F8D84301E00024CE
:105F800000BF00BF204670BD120E0020E80A0020AE
:105F90002DE9F05F81468A46934652464946A74816
:105FA000FFF7F0FA08B9BDE8F09FA548006800784F
:105FB000A2490978884200D0F5E74FF00008A148CF
:105FC000C0F800B09D48407806287CD004DC032847
:105FD00007D0042878D105E0102876D04128F9D1DF
:105FE0003BE000BF95484788007897490870934880
:105FF00040784870914800794006000E887000256E
:106000000FE03846FFF708FB0646310A6800C01C5F
:106010008D4A11546800001D1654781C87B2681C04
:10602000C5B286488088A842EBDC87488078C11CCE
:10603000854800F085FE044683488078C01C824A6B
:106040001454210A10468078001D1154104680789F
:10605000401D1146A1F80002CBE07848478800783F
:106060007949087075484078487074484088001233
:10607000887072488078C87070488088C0F3D710E4
:1060800008716E4800794006000E487100250FE047
:106090003846FFF7C1FA0646310A6800801D6A4A91
:1060A00011546800C01D1654781C87B2681CC5B214
:1060B00062488088A842EBDC604880884000801DF0
:1060C00081B2614802E018E08EE04BE000F038FE5B
:1060D00004465A4880884000801D5B4A1454210AB7
:1060E000564880884000C01D1154544880884000A4
:1060F00008301146A1F800027BE0504847888068CC
:1061000040784E498968097840EA01263146384688
:1061100000F0BAF88046B8F1000F00D06FE0082018
:106120004949A1F800024548007808704348407882
:106130004870424840880012887040488078C87093
:106140003E488068007808713C4880684078487113
:1061500006213D4800F0F4FD04463B498C71200ABD
:10616000C87144E035484788002517E03348806807
:1061700010F81560314881686800401C085C40EAEE
:1061800006263146384600F07FF88046781C87B2F4
:10619000B8F1000F00D032E0681CC5B227488088F3
:1061A000A842E3DC08202849A1F80002234800782F
:1061B0000870224840784870204840880012887053
:1061C0001E488078C8701D488088001208711B48DE
:1061D0000079487106211C4800F0B2FD04461A49B6
:1061E0008C71200AC87102E04FF0010807E000BF7F
:1061F00000BF1548B0F8001200F028F8D3E60520DB
:106200001149A1F800020D48007808700B48407849
:1062100040F080004870084680F80280032100F0BA
:106220008FFD04460849CC70200A08710846B0F872
:10623000001200F00BF800BFB5E60000204400207B
:10624000A0180020A41800202C44002070B504469B
:106250000D460A480A490968884204D12A4621465F
:10626000C36A984708E0074805490968884203D18E
:106270002A462146C36A984770BD0000DC09002009
:10628000A4180020200A002070B505460C46002600
:10629000B72D05D005DCA5F10C00AB2802D202E039
:1062A000BEE35BE1D1E18100794449688F4400009D
:1062B000D6030000D8030000DA030000DC0300006E
:1062C000DE030000E0030000E2030000E40300003E
:1062D000E6030000E80300000004000002040000E0
:1062E0000404000006040000A8040000C00400002C
:1062F000C2040000C4040000C6040000D80400006A
:10630000E4040000E6040000E8040000EA040000E1
:106310001C0500002E050000340500003A050000B1
:10632000400500004605000052050000540500002D
:1063300056050000580500006A05000082050000AF
:106340008405000086050000880500009C0500000B
:106350009E050000A0050000A2050000D405000075
:10636000D6050000D8050000DA050000EC050000A5
:10637000820A0000820A0000820A0000820A0000ED
:10638000820A0000820A0000820A0000820A0000DD
:10639000820A0000820A0000820A0000820A0000CD
:1063A000820A0000820A0000820A0000820A0000BD
:1063B000820A0000820A0000820A0000820A0000AD
:1063C000820A0000820A0000820A0000820A00009D
:1063D000820A0000820A0000820A0000820A00008D
:1063E000820A0000820A0000820A0000820A00007D
:1063F000820A0000820A0000820A0000820A00006D
:10640000820A0000820A0000820A0000820A00005C
:1064100022060000240600002606000028060000D0
:106420002A0600002C0600002E06000030060000A0
:106430003206000034060000360600003806000070
:1064400056060000580600005A0600005C060000D0
:106450005E060000600600006206000064060000A0
:1064600066060000680600006A0600006C06000070
:106470008A0600008C0600008E06000090060000D0
:1064800092060000940600009606000098060000A0
:106490009A0600009C0600009E060000A006000070
:1064A000BE060000C0060000C2060000C4060000D0
:1064B000C6060000C8060000CA060000CC060000A0
:1064C000CE060000D0060000D2060000D406000070
:1064D000F2060000F4060000F6060000F8060000D0
:1064E000FA060000FC060000FE060000000700009F
:1064F000020700000407000006070000080700006C
:1065000026070000280700002A0700002C070000CB
:106510002E0700003007000032070000340700009B
:1065200036070000380700003A0700003C0700006B
:106530005A0700005C0700005E07000060070000CB
:10654000620700006407000066070000680700009B
:106550006A0700006C0700006E070000F92D73D079
:1065600026DCA5F1B80041286FD2DFE800F0F1F099
:10657000EFEEEDECEBEAE9E8E7E6E5E4E3E2E1E0A3
:10658000DFDEDDDCDBDAD9D8D7D6D5D4D3D2D1D093
:10659000CFCECDCCCBCAC9C8C7C6C5C4C3C2C1C083
:1065A000BFBEBDBCBBBAB9B8B7B6B5B4B3B2B10023
:1065B000B5F58D7F7BD025DCA5F1FA002028D3D25C
:1065C000DFE810F0E002E102E202E302EE02EF0295
:1065D000F002F102F202FD02FE02FF0200030103DB
:1065E0000203030304030503060307030803090367
:1065F0000A030B030C030D030E030F031A032203FC
:106600002A03320340F22B11681A8D425CD015DC4C
:10661000A5F21B101028A7D2DFE810F00F0310031B
:1066200011031203130314031503160317031803AE
:10663000230324032503260327032803082844D023
:106640000EDC082890D201E09BE22FE0DFE810F09A
:106650002E001A031B031C031D031E032903310311
:106660000C2833D006DC092831D00A2871D00B2839
:106670001CD13AE30D286DD00E286CD0A0F2BD20BD
:106680000028F5D149E300BF00BF00BF00BF00BF35
:1066900000BF00BF00BF00BFA5F10C00FE4921F8FC
:1066A0001040A1F5F671D1F8E003804741E3C3E261
:1066B00000BF00BF00BFA5F11600F8490C54014609
:1066C000F5481430445434E3DBE2FAE20EE300E32D
:1066D00056E254E252E250E244E242E240E23EE25A
:1066E0003CE23AE238E236E234E232E230E224E2FC
:1066F00022E220E21EE21CE21AE218E20CE20AE2C6
:1067000008E206E204E202E200E2F7E1EEE1E5E19E
:10671000DCE1D0E1BFE1BDE1BBE1B9E1B7E1B5E169
:10672000B3E1B1E1AFE1ADE1ABE1A9E1A7E1A5E101
:10673000A3E1A1E19FE19DE19BE18BE189E187E19B
:1067400085E183E181E17FE17DE17BE179E177E151
:1067500075E1BFE2D5E2D5E22112D0480E3841758D
:1067600084752112CE4880F8081280F80942E0E2D0
:1067700000BF00BF00BFA5F11B01C8480A38445440
:10678000C5481E304454D4E2C6480484C448A0F826
:106790002242CEE200BF00BF00BFA5F12000BF4AE9
:1067A0000E3A14540146BC4818304454BE49486857
:1067B0008047BA490E39D1F830098047BA4948684C
:1067C0008047B749D1F8E0038047B2E24FF4FA605E
:1067D00094FBF0F100FB1140B4490880A9E2B349F1
:1067E0008C70A6E2B149CC70A3E2B0490C71A0E272
:1067F000AE494C719DE2AD498C710846C16888472D
:1068000097E200BF00BF00BFA5F12A00A8490C54C1
:106810000146A148223044548BE22112A4480E388C
:106820004175847521129E4880F8161280F817422F
:106830007FE200BF00BF00BFA5F12F009C490A39CD
:106840000C54014694482C30445472E200BF00BFFF
:1068500000BFA5F13300964A0E3A145401468E4803
:106860002630445490494868804791490E39D1F800
:10687000300980478C49486880478949D1F8E0034E
:10688000804756E200BF00BF00BFA5F1370188482E
:10689000093044548048303044544AE2211284483C
:1068A0000E38C176047721127D4880F8201280F8D6
:1068B00021427D49486880477D490E39D1F8300929
:1068C00080477949486880477549D1F8E003804797
:1068D0002FE200BF00BF00BF00BF00BF00BF00BF6E
:1068E00000BF00BF00BF00BF204604F069FB0146A7
:1068F000A5F1640268486A3020F812106849D1F89E
:10690000E003804715E200BF00BF00BF00BF00BF2B
:1069100000BF00BF00BF00BF00BF00BF204604F0A3
:106920004FFB0146A5F170025B48523020F812106F
:106930005B49D1F8E0038047FBE100BF00BF00BF27
:1069400000BF00BF00BF00BF00BF00BF00BF00BF4F
:10695000204604F035FB0146A5F17C024E48E230AA
:1069600020F812104E49D1F8E0038047E1E100BF62
:1069700000BF00BF00BF00BF00BF00BF00BF00BF1F
:1069800000BF00BF204604F01BFB0146A5F18802B2
:1069900041483A3020F812104149D1F8E0038047CD
:1069A000C7E100BF00BF00BF00BF00BF00BF00BF06
:1069B00000BF00BF00BF00BF204604F001FB01463E
:1069C000A5F194023448CA3020F812103449D1F8A5
:1069D000E0038047ADE100BF00BF00BF00BF00BFC4
:1069E00000BF00BF00BF00BF00BF00BF204604F0D3
:1069F000E7FA0146A5F1A0022748B23020F81210AC
:106A00002749D1F8E003804793E100BF00BF00BFF2
:106A100000BF00BF00BF00BF00BF00BF00BF00BF7E
:106A2000204604F0CDFA0146A5F1AC021A488230A6
:106A300020F812101A49D1F8E003804779E100BF2D
:106A400000BF00BF00BF00BF00BF00BF00BF00BF4E
:106A500000BF00BF204604F0B3FA0146A5F1B8021A
:106A60000D489A3020F812100D49D1F8E003804704
:106A70005FE100BF00BF00BF00BF00BF00BF00BF9D
:106A800000BF00BF00BF00BF00BF00BF00BF00BF0E
:106A900000BF00BF00BF0DE0D40C00205600002056
:106AA000E80A002058180020A80A0020C00A002088
:106AB000F60E002000BFA5F1C4019F4820F8114048
:106AC000A0F2E621D1F8E003804732E19B48A0F82C
:106AD0000E430146D1F8E00380472AE19748C0F809
:106AE00010430146D1F8E003804722E19348C0F803
:106AF00014430146D1F8E00380471AE18F48C0F8FB
:106B000018430146D1F8E003804712E100BF00BFFF
:106B100000BF00BF00BF00BFA5F1DC0186483630D2
:106B200020F811408549D1F8E003804701E100BF1A
:106B300000BF00BF00BF00BF00BFA5F1E3017E485A
:106B4000443020F811407D49D1F8E0038047F0E05F
:106B500000BF00BF00BF00BF00BF00BF00BF00BF3D
:106B600000BF00BFA5F1EA017348523020F8114080
:106B70007249D1F8E0038047DBE000BF00BF00BFEF
:106B800000BF00BF00BF00BF00BFA5F1F5016A480C
:106B9000683020F811406949D1F8E0038047C8E027
:106BA00000BF00BF00BF00BFA5F1FE0162487A3000
:106BB00020F811406149D1F8E0038047B9E000BFF7
:106BC00000BF00BF00BF00BF00BF00BF00BF00BFCD
:106BD00000BF00BF00BF00BF00BF00BF00BF00BFBD
:106BE00000BFA5F203115448843020F811405349E6
:106BF000D1F8E00380479CE05048A0F8904301465C
:106C0000D1F8E003804794E04C48A0F89243014655
:106C1000D1F8E00380478CE04848A0F8944301464F
:106C2000D1F8E003804784E04448A0F89643014649
:106C3000D1F8E00380477CE000BF00BF00BF00BF89
:106C400000BF00BF00BF00BF00BF00BFA5F58D7132
:106C50003948B23020F811403849D1F8E003804774
:106C600067E000BF00BF00BF00BF00BFA5F2251155
:106C70003148C83020F811403049D1F8E00380474E
:106C800057E000BF00BF00BF00BF00BFA5F22B113F
:106C90002948D43020F811402849D1F8E003804732
:106CA00047E02648A0F8C6430146D1F8E0038047F4
:106CB0003FE02248A0F8C8430146D1F8E0038047EE
:106CC00037E01E48A0F8CA430146D1F8E0038047E8
:106CD0002FE000BFA5F59A711748E63020F8114063
:106CE0001649D1F8E003804723E000BFA5F59B716A
:106CF0001148EA3020F811401049D1F8E0038047EC
:106D000017E000BFA5F59C710B48EE3020F811404C
:106D10000A49D1F8E00380470BE0084981F8D843DD
:106D2000D1F8E0038047054991F8D80306F0E2FA6C
:106D300000BF00BF304670BDCE0D0020E80A002025
:106D400030B502464FF6FF7012E012F8014B60407A
:106D5000002308E000F0010424B14AF2010484EAAF
:106D6000600000E040101C465D1CABB2082CF1DB5B
:106D70000C1EA1F10105A9B2E7D130BD00BFFEE7AD
:106D800010B503461446E01882B29A4205DD9142DE
:106D900001DA994207DA012010BD914203DB9942E2
:106DA00001DA0120F8E70020F6E70000154909881C
:106DB0000144144A1180144909880144124A11807F
:106DC000124909880144114A11800F490988B1F517
:106DD0007A7F07D300210C4A11800D490988491C8C
:106DE0000B4A11800949098842F21072914207D377
:106DF0000021064A118007490988491C054A11806B
:106E0000704700002C0000203200002034000020D9
:106E10002E0000203000002000201049088010497A
:106E200008801049088010490880084600880F49EA
:106E300008800D4800880E4908800B4800880D49DD
:106E40000880094800880C490880074800880B49D9
:106E50000880054800880A490880704732000020F1
:106E6000340000202E0000202C00002036000020DE
:106E7000380000203A0000203C0000203E000020A6
:106E8000400000207047000008B508490968C9089B
:106E90004FF47A72B1FBF2F14143009100BF00BFA1
:106EA00000994A1E00920029F9D108BD0C0000206B
:106EB0002DE9F04780460D462621404600F0C6F9F0
:106EC000064616B90020BDE8F08740F2B45086426D
:106ED00000DD06462821404600F0B8F90746B946CD
:106EE000C7F30A07002201213B48FCF76FFF384631
:106EF00000F022FA182101EB4811C8B200F012FA92
:106F000036480068C06800F0FF0AB819B0F5006F95
:106F100011DA00240CE0002000F004FA2F48006889
:106F2000C06800F0FF0A85F800A06D1C601C84B2E8
:106F3000B442F0DB3BE0C7F5006087B200240CE010
:106F4000002000F0EFF925480068C06800F0FF0A53
:106F500085F800A06D1C601C84B2BC42F0DB0122ED
:106F600011461D48FCF732FF002201211A48FCF7A8
:106F70002DFF002000F0E0F9182101EB4811C8B204
:106F800000F0D0F915480068C06800F0FF0A0CE076
:106F9000002000F0C7F911480068C06800F0FF0A3F
:106FA00085F800A06D1C601C84B2B442F0DB0122A5
:106FB00011460948FCF70AFF09EB06001FFA80F9A1
:106FC0004A462821404601F0F9F940220121404675
:106FD00001F0B4F9304676E7000C01407822002039
:106FE0002DE9F04780460D462621404600F064F921
:106FF000064616B90020BDE8F08740F2B45086423C
:1070000000DD06462821404600F056F90746B946FD
:10701000C7F30A0700224FF480513C48FCF7D6FE24
:10702000384600F09DF9182101EB4811C8B200F074
:107030008DF937480068C06800F0FF0AB819B0F54C
:10704000006F11DA00240CE0002000F07FF93048D6
:107050000068C06800F0FF0A85F800A06D1C601C85
:1070600084B2B442F0DB3CE0C7F5006087B2002494
:107070000CE0002000F06AF925480068C06800F0C4
:10708000FF0A85F800A06D1C601C84B2BC42F0DBD6
:10709000012211031D48FCF799FE00224FF4805194
:1070A0001A48FCF793FE002000F05AF9182101EB72
:1070B0004811C8B200F04AF915480068C06800F0ED
:1070C000FF0A0CE0002000F041F911480068C06898
:1070D00000F0FF0A85F800A06D1C601C84B2B44269
:1070E000F0DB012211030948FCF770FE09EB0600F2
:1070F0001FFA80F94A462821404601F07FF94022D4
:107100000121404601F03AF9304674E7000C014095
:10711000D022002070B50446002201210D48FCF762
:1071200055FE204600F008F9012000F0FBF80A485F
:107130000068C068C5B2002000F0F4F80648006896
:10714000C068C5B2012211460248FCF73FFE28463E
:1071500070BD0000000C01407822002070B504468C
:1071600000224FF480510D48FCF730FE204600F01D
:10717000F7F8012000F0EAF809480068C068C5B2D5
:10718000002000F0E3F806480068C068C5B201229C
:1071900011030248FCF71AFE284670BD000C01409E
:1071A000D022002070B504460D460022012110486F
:1071B000FCF70CFE284600F0BFF8082101EB441153
:1071C000C9B241F0010000F0ADF80A480068C0689B
:1071D000C6B2002000F0A6F806480068C068C6B233
:1071E000012211460248FCF7F1FD304670BD000057
:1071F000000C01407822002070B504460D460022A4
:107200004FF480510F48FCF7E1FD284600F0A8F844
:10721000082101EB4411C9B241F0010000F096F8D9
:1072200009480068C068C6B2002000F08FF8064820
:107230000068C068C6B2012211030248FCF7C6FD0F
:10724000304670BD000C0140D022002070B50546CC
:107250000E46002201211648FCF7B8FD304600F02A
:107260006BF8082101EB4511C9B241F0020000F0B2
:1072700059F810480068C06884B2002000F052F845
:107280000C480068C06884B2002000F04BF84FF64C
:10729000FF7000EA042407480068C068204484B2F4
:1072A000012211460248FCF791FD204670BD000006
:1072B000000C01407822002070B505460E460022E1
:1072C0004FF480511548FCF781FD304600F048F836
:1072D000082101EB4511C9B241F0020000F036F877
:1072E0000F480068C06884B2002000F02FF80C48F6
:1072F0000068C06884B2002000F028F84FF6FF70E4
:1073000000EA042406480068C068204484B20122D0
:1073100011030248FCF75AFD204670BD000C0140E5
:10732000D022002001B5FF23012269460148FDF764
:10733000B7FA08BD7822002010B504462012FFF7E6
:10734000F1FFE0B2FFF7EEFF10BD000001B5FF2333
:10735000012269460148FDF7A3FA08BDD0220020AA
:1073600010B504462012FFF7F1FFE0B2FFF7EEFF81
:1073700010BDF8B504460E461546334601220221DB
:107380002046009500F018F828B1606D40F020000C
:1073900060650320F8BD3346002280212046009519
:1073A00000F00AF828B1606D40F02000606503200D
:1073B000F0E70020EEE700002DE9F84F04460D4607
:1073C00090461E46DDF82890FCF706FDA0EB09006C
:1073D000371AFCF701FD82462C480068C0F3CB3019
:1073E0007843009045E0701C002842D0FCF7F4FC84
:1073F000A0EB0A00B84200D2A7BB2068406820F08A
:10740000E000216848606068B0F5827F0DD1A06817
:10741000B0F5004F03D0A068B0F5806F05D12068AB
:10742000006820F0400021680860A06AB0F5005FA5
:107430000DD100BF2068006820F40050216808606A
:107440002068006840F400502168086000BF0120F7
:1074500084F8510000BF002084F8500000BF0320D2
:10746000BDE8F88FFFE7009800B900270098401E9C
:107470000090206880682840A84201D1012000E0E7
:1074800000204045AFD10020EAE700000C000020BA
:10749000704710B5044601220021204600F04EFF3F
:1074A00001221146204600F049FF0520FCF706FAAC
:1074B00003212046FFF776FE132806D01022012173
:1074C000204600F03BFF002010BD04220121204691
:1074D00000F034FFFF20F7E710B504460122002139
:1074E000204600F04BFF01221146204600F046FFE7
:1074F0000520FCF7E3F903212046FFF77DFE132862
:1075000006D010220121204600F038FF002010BDD7
:1075100004220121204600F031FFFF20F7E710B5DB
:10752000044601220021204600F008FF01221146F6
:10753000204600F003FF0520FCF7C0F90321204698
:10754000FFF730FE132806D010220121204600F05C
:10755000F5FE002010BD02220121204600F0EEFEC3
:107560000520FCF7ABF903212046FFF71BFE14288A
:1075700006D010220121204600F0E0FE0020E9E7BD
:10758000FF20E7E710B5044601220021204600F065
:10759000F5FE01221146204600F0F0FE0520FCF722
:1075A0008DF903212046FFF727FE132806D010226D
:1075B0000121204600F0E2FE002010BD0222012140
:1075C000204600F0DBFE0520FCF778F90321204679
:1075D000FFF712FE142806D010220121204600F0E9
:1075E000CDFE0020E9E7FF20E7E710B504460222C0
:1075F0000021204600F0A2FE01221146204600F0A4
:107600009DFE0520FCF75AF903212046FFF7CAFD2D
:10761000222806D010220121204600F08FFE0020F3
:1076200010BDFF20FCE710B50446022200212046D1
:1076300000F0A4FE01221146204600F09FFE052026
:10764000FCF73CF903212046FFF7D6FD222806D09F
:1076500010220121204600F091FE002010BDFF20E5
:10766000FCE7000010B50120FFF7A0FB074801214F
:10767000826B904706480121826B904705480121A3
:10768000826B9047FCF7E6FB10BD0000DC09002090
:10769000200A0020640A002000B58FB0282105A828
:1076A000FBF778F914216846FBF774F90920059077
:1076B0004FF48030069000200790012009900B9035
:1076C00002200C90C1030D914FF4E0110E9105A81A
:1076D000FCF7D8FD08B1FBF767FE0F2000900220F1
:1076E0000190002002904FF48060039000200490ED
:1076F00002216846FCF7A2FC08B1FBF755FE0FB06B
:1077000000BD0000014802490860704700280008D9
:1077100008ED00E010B51048016C88470F48016C77
:1077200088470F48016C88470E49D1F834098047D3
:107730000D49D1F8340980470C49486980470B4905
:10774000886980470949C86980470949486880476E
:1077500005F050F910BD0000DC090020200A0020CF
:10776000640A002048000020E80E00202C180020A9
:10777000A80A00207047000010B5024988688047B9
:1077800010BD0000D40E002010B5074908698047DD
:107790000549486980470549D1F8380980470449B7
:1077A000D1F83809804710BDC00A002048000020E9
:1077B000E80E00207047704710B5044948688047BC
:1077C0000349D1F83C08804710BD00008C09002017
:1077D000081A0020704770B505466C6A0020E085E5
:1077E000E0842046FDF79BF970BD70B50646002584
:1077F000746A20684069C0F3C01594F841002128DC
:1078000005D125B10020E084204600F0FBF8206877
:107810004069C0F3801594F84200222805D125B1B3
:107820000020E085204600F0A7F8606C40F01000D2
:1078300060642046FDF773F970BD70B505466C6A4B
:107840002868006800F02000002842D1E08500BFD1
:1078500000BF21680C3151E8001F21F480702168BD
:107860000C3141E80002002AF3D100BF00BF00BF85
:107870002168143151E8001F21F001002168143102
:1078800041E80002002AF3D100BF00BF00BF216819
:10789000143151E8001F21F040002168143141E803
:1078A0000002002AF3D100BF202084F84200206BA0
:1078B00001280ED100BF00BF21680C3151E8001F24
:1078C00021F0100021680C3141E80002002AF3D1B8
:1078D00000BF00206063206B012804D1A18D2046E9
:1078E000FDF7D7F802E02046FDF750FC70BD70B5FB
:1078F00005466C6A01206063206B012805D1A08DCC
:1079000041082046FDF7C5F802E02046FDF73FFCA0
:1079100070BD70B505466C6A2868006800F02000EC
:10792000F8B90020E08400BF00BF2168143151E89D
:10793000001F21F080002168143141E80002002A74
:10794000F3D100BF00BF00BF21680C3151E8001F18
:1079500041F0400021680C3141E80002002AF3D1D7
:1079600002E02046FDF75AFC70BD70B50446656A1A
:107970002846FDF779FC70BD00BF00BF02680C32DD
:1079800052E8002F22F4907102680C3242E8001392
:10799000002BF3D100BF00BF00BF0268143252E8D1
:1079A000002F22F001010268143242E80013002B7C
:1079B000F3D100BF016B01290ED100BF00BF0268E7
:1079C0000C3252E8002F22F0100102680C3242E81B
:1079D0000013002BF3D100BF202180F842100021BA
:1079E0000163704710B504462068C06820F040006D
:1079F0002168C860202084F841002046FDF70EFC75
:107A0000002010BD00BF00BF02680C3252E8002FFA
:107A100022F0C00102680C3242E80013002BF3D1BF
:107A200000BF202180F841107047F8B5044694F853
:107A30004200222875D1A068B0F5805F0CD1206982
:107A400050B90025A66A20684068C0F3080030805D
:107A5000A06A801CA06215E0A56A0026A068B0F5A7
:107A6000805F03D0A06828B9206918B920684068F1
:107A7000287004E02068406800F07F002870A06A49
:107A8000401CA062E08D401E80B2E085002846D1F7
:107A90002068C06820F020002168C8602068C068A5
:107AA00020F480702168C8602068406920F00100DF
:107AB00021684861202084F8420000206063206B28
:107AC000012826D10020206300BF00BF21680C31AF
:107AD00051E8001F21F0100021680C3141E800023C
:107AE000002AF3D100BF2068006800F010001028C1
:107AF0000AD100BF00200090206800680090206834
:107B00004068009000BF00BFA18D2046FCF7C1FF78
:107B100002E02046FDF73AFB0020F8BD01E000201E
:107B2000FBE70220F9E7000070B504462168096907
:107B300021F44051E2681143226811612269A16871
:107B40001143626941EA02052168C96841F20C6289
:107B5000914329432268D1602168496921F4407129
:107B6000A2691143226851612D4A2168914202D1D4
:107B7000FCF740FB01E0FCF72DFB00EBC00101EB43
:107B8000001162689200B1FBF2F100EBC00202EB5F
:107B9000001263689B00B2FBF3F26423B2FBF3F2C2
:107BA00002EBC20303EB0212A1EB8201322202EBD1
:107BB00001116422B1FBF2F101F0F00100EBC0020F
:107BC00002EB001263689B00B2FBF3F26423B2FB8A
:107BD000F3F201EB021200EBC00101EB001163684C
:107BE0009B00B1FBF3F100EBC00303EB00136668ED
:107BF000B600B3FBF6F36426B3FBF6F303EBC30660
:107C000006EB0313A1EB8301322303EB0111642381
:107C1000B1FBF3F101F00F0111442268916070BDD6
:107C20000038014077B581B0044615460298A0623D
:107C3000A58500206064222084F842002848E16B7A
:107C400088622848E16BC8622748E16B086300201E
:107C5000E16B486302AE32682368191D2B46E06B66
:107C6000FBF7DEFD00BF0020009020680068009058
:107C700020684068009000BF00BF206970B100BF5D
:107C800000BF21680C3151E8001F41F48070216869
:107C90000C3141E80002002AF3D100BF00BF00BF51
:107CA0002168143151E8001F41F0010021681431AE
:107CB00041E80002002AF3D100BF00BF00BF2168E5
:107CC000143151E8001F41F040002168143141E8AF
:107CD0000002002AF3D100BF002004B070BD0000F4
:107CE0003B780008EF780008EB770008014691F830
:107CF0004100212828D18868B0F5805F0BD1086940
:107D000048B90A6A1088C0F308000B685860086A0E
:107D1000801C086205E00B6A581C086218780B6822
:107D20005860C88C401E80B2C88458B90868C068C2
:107D300020F080000B68D8600868C06840F0400000
:107D40000B68D860002070470220FCE708B50D489A
:107D50000068006800F0100010280FD100BF00205C
:107D60000090084800680068009006480068406875
:107D7000009000BF00BF0448416B88470148FCF7F2
:107D8000CFFE08BD28230020DC09002008B50D48DF
:107D90000068006800F0100010280FD100BF00201C
:107DA0000090084800680068009006480068406835
:107DB000009000BF00BF0448416B88470148FCF7B2
:107DC000AFFE08BD70230020200A002008B50D4832
:107DD0000068006800F0100010280FD100BF0020DC
:107DE00000900848006800680090064800684068F5
:107DF000009000BF00BF0448416B88470148FCF772
:107E00008FFE08BDB8230020640A002000BFFEE7F3
:107E100010B5002210210748FBF7D8FF3220FBF7EE
:107E20004DFD012210210348FBF7D0FF6420FBF732
:107E300045FD10BD0008014010B500224FF400615F
:107E40000748FBF7C3FF3220FBF738FD0122D102C0
:107E50000348FBF7BBFF6420FBF730FD10BD0000BB
:107E6000000801403EB500240020009001900290DF
:107E7000802100F0FBF90A20FBF720FD04223348A3
:107E80000168012000F034FB042230480168091D1C
:107E9000052000F02DFB2E48006800902C48001DA6
:107EA000006801902A480830006802900198000A92
:107EB0002649096808720198C1B2244800684172D5
:107EC0000298010E2148006881720298010C1F4837
:107ED0000068C1720298010A1C4800680173029888
:107EE000C1B21A480068417318480068007A00F06F
:107EF000FE0040F002001549096808720622134886
:107F000001680831092000F0F3FA04220F480168E3
:107F10000E310F2000F0ECFA00BF0BE0E0B20222BD
:107F20001E2100F00BFAE0B202221F2100F006FA37
:107F3000601C84B2082CF1DB4FF4FA61192000F0C8
:107F4000C9F908211B2000F091F93EBD88090020E5
:107F5000E8F7FF1F3EB5002400200090019002903A
:107F6000802100F09DF90A20FBF7A8FC0422344888
:107F70000168012000F0E0FA042231480168091D7F
:107F8000052000F0D9FA2F48006800902D48001D08
:107F90000068401C01902B4808300068401C02908B
:107FA0000198000A2649096808720198C1B224485C
:107FB000006841720298010E21480068817202989F
:107FC000010C1F480068C1720298010A1C48006831
:107FD00001730298C1B21A480068417318480068DA
:107FE000007A00F0FE0040F00200154909680872AE
:107FF0000622134801680831092000F09DFA042286
:108000000F4801680E310F2000F096FA00BF0BE018
:10801000E0B202221E2100F0B1F9E0B202221F21DB
:1080200000F0ACF9601C84B2082CF1DB4FF4FA616B
:10803000192000F069F908211B2000F031F93EBD3C
:1080400028180020E8F7FF1F2DE9F04704460E46E8
:10805000904620780021FFF7A5F800F00F002228B5
:108060000DD0207804F109020C2100F0E7F9A37B80
:10807000617B43EA01222078102100F09FF92078EB
:108080002421FFF7E3F80746B946C7F30A070022A1
:1080900001213048FBF79AFE3846FFF74DF9217869
:1080A000102202EB4111C9B241F00400FFF73AF986
:1080B00007EB0800B0F5006F0ADA002505E016F8B6
:1080C000010BFFF72FF9681C85B24545F7DB2BE064
:1080D000C7F5006087B2002505E016F8010BFFF731
:1080E00021F9681C85B2BD42F7DB0122114619480F
:1080F000FBF76CFE002201211648FBF767FE00200B
:10810000FFF71AF92178102202EB4111C9B241F0B0
:108110000400FFF707F905E016F8010BFFF702F975
:10812000681C85B24545F7DB012211460948FBF77B
:108130004DFE09EB08001FFA80F920784A462421F9
:1081400000F03CF920782022012100F0F7F8BDE88A
:10815000F0870000000C01402DE9F04704460E4670
:10816000904620780021FFF747F800F00F00222802
:108170000DD0207804F109020C2100F08BF9A37BCB
:10818000617B43EA01222078102100F037F9207842
:108190002421FFF791F80746B946C7F30A070022E2
:1081A0004FF480513048FBF711FE3846FFF7D8F8FE
:1081B0002178102202EB4111C9B241F00400FFF70F
:1081C000C5F807EB0800B0F5006F0ADA002505E0F6
:1081D00016F8010BFFF7BAF8681C85B24545F7DBC6
:1081E0002CE0C7F5006087B2002505E016F8010B0A
:1081F000FFF7ACF8681C85B2BD42F7DB0122110322
:108200001948FBF7E3FD00224FF480511648FBF7B5
:10821000DDFD0020FFF7A4F82178102202EB4111C8
:10822000C9B241F00400FFF791F805E016F8010B20
:10823000FFF78CF8681C85B24545F7DB0122110376
:108240000948FBF7C3FD09EB08001FFA80F9207805
:108250004A46242100F0D2F820782022012100F0A3
:108260008DF8BDE8F0870000000C014070B50546B0
:108270000C46002201210948FBF7A8FD2846FFF71C
:108280005BF80520FFF74EF82046FFF74BF8012278
:1082900011460248FBF79AFD70BD0000000C01403A
:1082A00070B505460C4600224FF480510848FBF794
:1082B0008DFD2846FFF754F80520FFF747F82046C4
:1082C000FFF744F8012211030148FBF77FFD70BD61
:1082D000000C014070B505460C46002201210948FA
:1082E000FBF774FD2846FFF727F80620FFF71AF87A
:1082F0002046FFF721F8012211460248FBF766FDF0
:1083000070BD0000000C014070B505460C4600220F
:108310004FF480510848FBF759FD2846FFF720F835
:108320000620FFF713F82046FFF71AF80122110381
:108330000148FBF74BFD70BD000C014070B50446D1
:108340000D461646002201210B48FBF73FFD28464B
:10835000FEF7F2FF082101EB4411C9B241F005001C
:10836000FEF7E0FF3046FEF7DDFF0122114602482E
:10837000FBF72CFD70BD0000000C014070B50446F9
:108380000D46164600224FF480510B48FBF71EFDA8
:108390002846FEF7E5FF082101EB4411C9B241F080
:1083A0000500FEF7D3FF3046FEF7D0FF0122110390
:1083B0000148FBF70BFD70BD000C014070B5044691
:1083C0000D461646002201210B48FBF7FFFC28460C
:1083D000FEF7B2FF082101EB4411C9B241F00600DB
:1083E000FEF7A0FF3046FEF7A7FF01221146024824
:1083F000FBF7ECFC70BD0000000C014070B50446BA
:108400000D46164600224FF480510B48FBF7DEFC68
:108410002846FEF7A5FF082101EB4411C9B241F03F
:108420000600FEF793FF3046FEF79AFF0122110384
:108430000148FBF7CBFC70BD000C014070B5054650
:108440000E461446002201211148FBF7BFFC3046BE
:10845000FEF772FF082101EB4511C9B241F0070098
:10846000FEF760FF14F8010BFEF75CFF14F8010B38
:10847000FEF758FF14F8010BFEF754FF14F8010B38
:10848000FEF750FF012211460148FBF79FFC70BD2B
:10849000000C014070B505460E46144600224FF40C
:1084A00080511248FBF792FC3046FEF759FF082135
:1084B00001EB4511C9B241F00700FEF747FF14F880
:1084C000010BFEF743FF14F8010BFEF73FFF14F812
:1084D000010BFEF73BFF14F8010BFEF737FF0122FB
:1084E00011030248FBF772FC70BD0000000C014054
:1084F0002DE9F04107460C461546002201210D48A2
:10850000FBF764FC3846FEF717FF0420FEF70AFF6E
:10851000002605E014F8010BFEF704FF701C86B27C
:10852000AE42F7DB012211460248FBF74FFCBDE8E3
:10853000F0810000000C01402DE9F04107460C4697
:10854000154600224FF480510C48FBF73FFC38469B
:10855000FEF706FF0420FEF7F9FE002605E014F8FA
:10856000010BFEF7F3FE701C86B2AE42F7DB012270
:1085700011030248FBF72AFCBDE8F081000C014022
:108580000FB4054B10B503A9044A029800F022F974
:1085900010BC5DF814FB0000E1A90008682200206F
:1085A0000FB41CB50246002007AC00290BD0491EB1
:1085B000CDE90021054B6A462146069800F00AF9EC
:1085C000009A002111701CBC5DF814FB038F000899
:1085D0000FB4084B10B504A902AA039800F0FAF8EA
:1085E000044602A9002000F097FC204610BC5DF86C
:1085F00014FB0000198F000802480068C0F3022035
:10860000704700000CED00E010B5002804DB0A07FD
:10861000130E054A135406E00A07140E034A00F02D
:108620000F031B1FD45410BD00E400E018ED00E060
:1086300002E008C8121F08C1002AFAD1704770472B
:10864000002001E001C1121F002AFBD17047000089
:108650002DE9FF5F82B00021DDE90430020DDDF875
:1086600040B0034318D044F61050A2F2FF32424308
:108670001514119801281FD0A5EB0B00401C5FEAD0
:10868000000A4FF000064E4FDFF83891B0465046D2
:1086900015D5CAF1000413E0119801244AA301285A
:1086A00001D16FEA0B010298119AC0E90031C0E9CB
:1086B000024206B0BDE8F09FCBF10000DFE70446C0
:1086C0000021404A491842EB0450CDE9001012E065
:1086D000E00707D032463B4640464946FAF7ACFA37
:1086E0008046894632463B4610461946FAF7A4FAB8
:1086F00006460F466410002CEAD1DDE90401DDE9ED
:108700000023BAF1000F06DAFAF796FA42464B4612
:10871000FAF792FA05E0FAF701FB42464B46FAF700
:10872000FDFA04460E460022284BFAF77FFB03D8D9
:108730004FF0FF30014607E00022254B204631462E
:10874000FAF7D3F9FAF759FB102409E0002C0ADBF9
:108750000A220023FAF798F9039B30321A55641E57
:1087600050EA0102F2D1641C039AC4F111031444CB
:10877000119A012A03D0012208430DD10AE00843CF
:1087800004D000204FF0110B119072E7A3EB0B0502
:108790006D1E0DE05B4504DD4FF0000205F10105A3
:1087A00004E003DA4FF00002A5F10105002AECD045
:1087B00002981199C0E90231C0E9004579E700004B
:1087C000000014400000F03F300000000000F043C3
:1087D0000000E03F2DE9FF4F95B09B4689460646D5
:1087E00000250FE2252877D100242746F84A0121E9
:1087F000059400E0044316F8013F203B01FA03F022
:108800001042F7D130782A2811D06FF02F0330783A
:10881000A0F13002092A16D8059A44F0020402EBAE
:10882000820203EB42021044761C0590EFE759F8F0
:10883000042B0592002A03DA504244F400540590B8
:1088400044F00204761C30782E2816D116F8010F59
:1088500044F004042A280DD06FF02F023078A0F1E4
:108860003003092B09D807EB870302EB4303C71832
:10887000761CF3E759F8047B761C30786C280FD00F
:1088800006DC4C2817D068280DD06A2814D104E0E3
:10889000742810D07A280FD10DE044F400140AE0B7
:1088A00044F4801401E044F440147278824202D10E
:1088B00004F58014761C761C307866280BD013DC07
:1088C000582877D009DC002875D04528F6D04628EE
:1088D000F4D047281AD19DE118E0632835D06428E8
:1088E00079D0652812D195E1702873D008DC67280B
:1088F000F1D069286FD06E280DD06F2806D1B5E071
:1089000073282CD0752875D0782874D05A461799BA
:1089100090476D1C75E1C4F30250022809D003286A
:108920000DD0D9F8001004280DD00D6009F104090C
:1089300067E1D9F80010EA17C1E90052F6E7D9F863
:1089400000100D80F2E70D70F0E719F8041B8DF8A8
:10895000001000208DF80100EA46012003E059F8DC
:1089600004AB4FF0FF3061074FF0000102D40DE07F
:1089700008F101018846B9420FDA8045F8DB1AF8A0
:1089800008100029F4D108E008F10101884681426D
:10899000FADB1AF808100029F6D105985B46A0EB1F
:1089A000080721463846179A00F094FA284400EB4D
:1089B000080507E04DE029E10DE01AF8010B5A46E1
:1089C00017999047B8F10108F7D25B46214638461F
:1089D000179A13E142E00A220092C4F302524FF0C8
:1089E000000A022A08D059F804CB032A4FEAEC7196
:1089F0000AD00DE029E02AE009F1070121F0070281
:108A0000F2E802C1914609E00FFA8CFC4FEAEC71E2
:108A1000042A03D14FFA8CFC4FEAEC71002907DAE3
:108A20000A460021DCF1000C61EB02012D2202E07C
:108A3000220504D52B228DF80420012203E0E20751
:108A400001D02022F7E7904659E00A2102E01022E7
:108A50000DE010214FF0000A00910BE010224FF0C2
:108A6000000A44F004040827009203E008224FF0B3
:108A7000000A0092C4F30252022A05D059F804CB2E
:108A80000021032A08D009E009F1070121F00702BB
:108A9000F2E802C1914605E01FFA8CFC042A01D1DC
:108AA0000CF0FF0C4FF00008220728D5702806D0E4
:108AB000009B83F0100353EA0A0305D00EE0402226
:108AC0008DF80420012208E05CEA010206D0302281
:108AD0008DF804208DF8050002229046009B83F05B
:108AE000080353EA0A030AD15CEA010201D16207D2
:108AF00005D530228DF804204FF001087F1E58283C
:108B000004D034A003900EA802900DE036A0F9E73F
:108B100053466046009AF9F7B7FF84460398825C93
:108B20000298401E029002705CEA0100F0D10298A7
:108B300006A9081A00F1200A600702D524F480343F
:108B400000E00127574502DDA7EB0A0000E0002006
:108B500000EB0A01009005984144401A0590E0039B
:108B600006D45B462146179A059800F0B3F90544F0
:108B7000002706E001A85A46C05D179990476D1C72
:108B80007F1C4745F6DBE0030CD55B462146179A70
:108B9000059800F09FF9054404E030205A461799E3
:108BA00090476D1C0099481E00900029F5DC08E0F4
:108BB000029802995A460078491C029117999047E9
:108BC0006D1CBAF10001AAF1010AF1DC65E10000B7
:108BD0000928010030313233343536373839616293
:108BE0006364656600000000303132333435363757
:108BF00038394142434445460000000000F058F92E
:108C00000544761C307800287FF4ECAD19B0284676
:108C1000BDE8F08F620700D4062709F1070222F0B1
:108C2000070CFCE80223E14603F000485FEA080C69
:108C300002D00FF2702C0DE05FEA045C02D50FF257
:108C4000682C07E05FEAC47C02D00FF2602C01E0E0
:108C5000AFF2700C4FF0FF3823F00043CDF850C056
:108C600065280CD006DC452809D046281DD04728A9
:108C70003DD13DE0662818D067287ED138E000213C
:108C8000112F01DB112000E0781CCDE9000106A9BD
:108C90000EA8FFF7DDFCDDE90F010E9A039100211C
:108CA000009207F1010A04914DE04FF00040009757
:108CB000CDE9011006A90EA8FFF7CAFCDDE90F02F5
:108CC00003920E9B11990022DDF80CA000930492F0
:108CD00011B9791C00EB010AB7EB0A0004D4C0F10A
:108CE000FF3007F1010A0490AAEB0700019044E06D
:108CF000012F00DA01270021112F01DD112000E0F2
:108D00003846CDE9000106A90EA8FFF7A1FCDDE970
:108D10000F010E9A0391002104910092BA46210797
:108D20000CD40399514500DA8A46BAF1010F05DDEA
:108D3000009AAAF10101515C302908D0B84202DA48
:108D400010F1040F06DA0121CDE9011015E0AAF1B6
:108D50000101E9E7002805DC049901440491AAEB2C
:108D6000000102E0411C514500DD8A460499401A89
:108D7000401C01904FF000400290200704D401985D
:108D8000504501DBCDF8048000208DF84F0002989B
:108D90000DF14F07B0F1004F25D02B200E90029817
:108DA0004FF0020800280CDA404202902D200E906D
:108DB00007E00A210298F9F751FE3031029007F8D6
:108DC000011DB8F10001A8F10108F2DC02980028A9
:108DD000EFD1791E0E980870307800F0200040F036
:108DE000450007F8020D12A8C01B00F107081498EF
:108DF000007800B1012000EB0A01019801EBE0715D
:108E000005984144401A401E0590E00306D45B4695
:108E10002146179A059800F05DF8054414980078EB
:108E200018B15A46179990476D1CE00324D55B464C
:108E30002146179A059800F04DF805441CE0049867
:108E4000002807DBDDE90301884203DD0098405C70
:108E5000179901E0179930205A469047049805F178
:108E60000105401C04900198401E019004D12E2061
:108E70005A46179990476D1CBAF10001AAF1010AF0
:108E8000DDDC05E017F8010B5A46179990476D1C79
:108E9000B8F10001A8F10108F4DC5B462146179AFD
:108EA0000598ABE62D0000002B000000200000001C
:108EB0002DE9F041044600251E461746880404D4D7
:108EC00005E039462020B0476D1C641EF9D52846C0
:108ED000BDE8F0812DE9F041044600251E4690468C
:108EE000C80301D5302700E02027880404D505E019
:108EF00041463846B0476D1C641EF9D52846BDE88A
:108F0000F0814A68002A06D00A68531C0B60107072
:108F10004868401E486070470A68531C0B60107018
:108F200070470146080240EA212080B270470000E5
:108F30001FB5402000900020019002900320039074
:108F400069460248FAF7A0FD1FBD0000000C014071
:108F50001FB54020009001200190002002900320C6
:108F6000039069460148FAF78FFD1FBD000C0140D0
:108F700010B5012280212148FAF728FF0022202184
:108F80001E48FAF723FF00F057F91D4800680088D3
:108F9000632818DC1A48006880780C2813DC18480D
:108FA0000068C0781F280EDC154800680079172873
:108FB00009DC1348006840793B2804DC104800684D
:108FC00080793B2818DD19200D49096808800120A7
:108FD0000B49096888700A490968C8700020084967
:108FE0000968087106490968487105490968887166
:108FF0000348006800F074F810BD0000000C014048
:10900000E40A002010B5FAF7E7FE05490968441A9A
:109010004FF47A70B4FBF0F002490968084410BDBF
:10902000BC0A0020B80A00202DE9F0438DB00546A7
:109030000E460DB1112E02DA0DB0BDE8F083FAF73D
:10904000CBFE1D490968441A4FF47A70B4FBF0F066
:109050001A49096847184FF47A70B4FBF0F100FB25
:10906000114807A808A909AA0AABCDE90021029076
:109070000BAA0CA9384603F095FE0A20B8FBF0F0C5
:1090800000F0FF099DF81C009DF820109DF8242099
:10909000CDE90409CDE902219DF828009DF82C10A6
:1090A000CDE90010BDF8303005A231462846FFF763
:1090B00077FA00BFC0E70000BC0A0020B80A002011
:1090C00025303464253032642530326425303264F2
:1090D00025303264253032642530326400000000CF
:1090E00070B50446208863280EDCA0780C280BDCC1
:1090F000E0781F2808DC2079172805DC60793B28F8
:1091000002DCA0793B2801DD002070BD00218E200B
:1091100000F080FA8021084600F07CFA2078FCF705
:10912000A6F8054629468C2000F074FAA078FCF7D2
:109130009EF805462946882000F06CFAE078FCF796
:1091400096F805462946862000F064FA2079FCF757
:109150008EF805462946842000F05CFA6079FCF719
:1091600086F805462946822000F054FAA079FCF7DB
:109170007EF805462946802000F04CFA80218E209A
:1091800000F048FA0120C0E72DE9FF5F04460D46D4
:1091900016461F46DDE90F9ADDF83880B4F5FA6F00
:1091A00016DB40F63300844212DC012D10DB0C2D5F
:1091B0000EDC012E0CDB1F2E0ADC172F08DCB8F1A9
:1091C0003B0F05DCB9F13B0F02DCBAF1630F03D9A9
:1091D000002004B0BDE8F09FA4F5FA6080B2ADF8BD
:1091E00008008DF80A508DF80B608DF80C708DF822
:1091F0000D808DF80E9002A8FFF772FF012801D0B4
:109200000020E6E70AEB8A004FEA400B3B46324675
:1092100029462046CDE9008901F046FB0449086053
:10922000FAF7DAFDA0EB0B00024908600120D0E755
:10923000B80A0020BC0A002010B58C2000F0AAF863
:1092400004462046E21704EB12721211A4EB02123C
:109250002146E31704EB13731B1103EB830302EBAB
:1092600043023B4B1B681A80882000F093F80446A9
:109270002046E21704EB12721211A4EB02122146EF
:10928000E31704EB13731B1103EB830302EB43029D
:109290002F4B1B689A70862000F07CF8044620460D
:1092A000E21704EB12721211A4EB02122146E3172B
:1092B00004EB13731B1103EB830302EB4302244BF8
:1092C0001B68DA70842000F065F804462046E21737
:1092D00004EB12721211A4EB02122146E31704EB05
:1092E00013731B1103EB830302EB4302184B1B6840
:1092F0001A71822000F04EF804462046E21704EB73
:1093000012721211A4EB02122146E31704EB13733D
:109310001B1103EB830302EB43020D4B1B685A71D5
:10932000802000F037F804462046E21704EB127262
:109330001211A4EB02122146E31704EB13731B1165
:1093400003EB830302EB4302014B1B689A7110BDD0
:10935000E40A00201CB50C48008800F5FA6084B2CD
:109360000948807908494979CDE900100648037910
:10937000C2788178204601F097FA04490860FAF72C
:109380002BFD034908601CBDC00A0020B80A00205C
:10939000BC0A002070B50546012280219C48FAF7DE
:1093A00015FD00BF00BF00BF00BF00BF00BF00BF72
:1093B00000BF00BF00BF00BF00BF00BF00BF00BFB5
:1093C00000BF00BF00BF00BF00BF00BF00BF00BFA5
:1093D00000BF00BF00BF00BF00BF00BF00BF45F01F
:1093E0000105002474E005F0010028B101224021AC
:1093F0008748FAF7EBFC04E0002240218448FAF7A2
:10940000E5FC00BF00BF00BF00BF00BF00BF00BF42
:1094100000BF00BF00BF00BF00BF00BF00BF00BF54
:1094200000BF00BF00BF00BF00BF00BF00BF00BF44
:1094300000BF00BF00BF00BF00BF00BF00BF0122D0
:1094400020217348FAF7C2FC00BF00BF00BF00BF75
:1094500000BF00BF00BF00BF00BF00BF00BF00BF14
:1094600000BF00BF00BF00BF00BF00BF00BF00BF04
:1094700000BF00BF00BF00BF00BF00BF00BF00BFF4
:1094800000BF00BF002220216148FAF79FFC00BF07
:1094900000BF00BF00BF00BF00BF00BF00BF00BFD4
:1094A00000BF00BF00BF00BF00BF00BF00BF00BFC4
:1094B00000BF00BF00BF00BF00BF00BF00BF00BFB4
:1094C00000BF00BF00BF00BF00BF6D10601CC4B272
:1094D000082C88DBFFF72CFD002470E0761040217B
:1094E0004B48FAF761FC10B146F0800601E006F047
:1094F0007F0600BF00BF00BF00BF00BF00BF00BFAE
:1095000000BF00BF00BF00BF00BF00BF00BF00BF63
:1095100000BF00BF00BF00BF00BF00BF00BF00BF53
:1095200000BF00BF00BF00BF00BF00BF00BF0122DF
:1095300020213748FAF74AFC00BF00BF00BF00BF38
:1095400000BF00BF00BF00BF00BF00BF00BF00BF23
:1095500000BF00BF00BF00BF00BF00BF00BF00BF13
:1095600000BF00BF00BF00BF00BF00BF00BF00BF03
:1095700000BF00BF002220212548FAF727FC00BFCA
:1095800000BF00BF00BF00BF00BF00BF00BF00BFE3
:1095900000BF00BF00BF00BF00BF00BF00BF00BFD3
:1095A00000BF00BF00BF00BF00BF00BF00BF00BFC3
:1095B00000BF00BF00BF00BF00BF601CC4B2082CCA
:1095C0008CDB002280211248FAF700FC00BF00BFAC
:1095D00000BF00BF00BF00BF00BF00BF00BF00BF93
:1095E00000BF00BF00BF00BF00BF00BF00BF00BF83
:1095F00000BF00BF00BF00BF00BF00BF00BF00BF73
:1096000000BF00BF00BF00BFFFF7A2FC304670BD27
:10961000000C014070B505460E46012280219C4891
:10962000FAF7D4FB00BF00BF00BF00BF00BF00BF00
:1096300000BF00BF00BF00BF00BF00BF00BF00BF32
:1096400000BF00BF00BF00BF00BF00BF00BF00BF22
:1096500000BF00BF00BF00BF00BF00BF00BF00BF12
:1096600005F0FE05002474E005F0010028B1012298
:1096700040218748FAF7AAFB04E0002240218448F1
:10968000FAF7A4FB00BF00BF00BF00BF00BF00BFD0
:1096900000BF00BF00BF00BF00BF00BF00BF00BFD2
:1096A00000BF00BF00BF00BF00BF00BF00BF00BFC2
:1096B00000BF00BF00BF00BF00BF00BF00BF00BFB2
:1096C000012220217248FAF781FB00BF00BF00BFD2
:1096D00000BF00BF00BF00BF00BF00BF00BF00BF92
:1096E00000BF00BF00BF00BF00BF00BF00BF00BF82
:1096F00000BF00BF00BF00BF00BF00BF00BF00BF72
:1097000000BF00BF00BF002220216148FAF75EFBC6
:1097100000BF00BF00BF00BF00BF00BF00BF00BF51
:1097200000BF00BF00BF00BF00BF00BF00BF00BF41
:1097300000BF00BF00BF00BF00BF00BF00BF00BF31
:1097400000BF00BF00BF00BF00BF00BF6D10601CA6
:10975000C4B2082C88DB002474E006F0010028B1B4
:10976000012240214A48FAF731FB04E0002240215F
:109770004748FAF72BFB00BF00BF00BF00BF00BF88
:1097800000BF00BF00BF00BF00BF00BF00BF00BFE1
:1097900000BF00BF00BF00BF00BF00BF00BF00BFD1
:1097A00000BF00BF00BF00BF00BF00BF00BF00BFC1
:1097B00000BF012220213648FAF708FB00BF00BF96
:1097C00000BF00BF00BF00BF00BF00BF00BF00BFA1
:1097D00000BF00BF00BF00BF00BF00BF00BF00BF91
:1097E00000BF00BF00BF00BF00BF00BF00BF00BF81
:1097F00000BF00BF00BF00BF002220212448FAF7AD
:10980000E5FA00BF00BF00BF00BF00BF00BF00BF40
:1098100000BF00BF00BF00BF00BF00BF00BF00BF50
:1098200000BF00BF00BF00BF00BF00BF00BF00BF40
:1098300000BF00BF00BF00BF00BF00BF00BF761069
:10984000601CC4B2082C88DB002280211048FAF783
:10985000BDFA00BF00BF00BF00BF00BF00BF00BF18
:1098600000BF00BF00BF00BF00BF00BF00BF00BF00
:1098700000BF00BF00BF00BF00BF00BF00BF00BFF0
:1098800000BF00BF00BF00BF00BF00BF00BF70BD72
:10989000000C014010B586B00446002001900290F3
:1098A00004940120059001A902A8FAF71BF806B05C
:1098B00010BD000010B50649486880474FF4F672A5
:1098C0000449054800F0B2F901494868804710BDD5
:1098D000A80A0020D40C002000FC000810B54FF4AA
:1098E000F6720F49A1F5F670F9F780F8B8B10D4995
:1098F0004868804772B64FF4F67209490A4800F08A
:10990000B9F9044634B94FF4F6720549A1F5F67079
:10991000F9F727F862B603494868804700BF10BDD1
:10992000D40C0020A80A002000FC000870B541F209
:109930008A340A21354880F80012152180F8011276
:10994000362180F80212022180F80312211280F8D9
:10995000081280F80942FF2180F80A1280F80B12E1
:10996000FC2180F80C12002180F80D120A2180F8E9
:109970000412152180F80512342180F80612012105
:1099800080F807120021A0F82212A51E4FF4FB76E2
:10999000C02180F80E12A82180F80F12642180F8EF
:1099A0001012672180F81112291280F8161280F81F
:1099B0001752FF2180F8181280F8191280F81A1235
:1099C000002180F81B12C02180F81212A82180F813
:1099D0001312642180F81412012180F81512C0219D
:1099E00080F81C12A82180F81D12642180F81E1234
:1099F0003D2180F81F12311280F8201280F8216278
:109A00000021A0F82412FFF769FF70BDE80A0020CA
:109A100010B5FFF74FFF804890F80002FF2810D1E3
:109A20007D4890F80102FF280BD17B4890F8020294
:109A3000FF2806D1784890F80302FF2801D1FFF7EC
:109A400075FF7548B0F83E024FF6FF7188422ED17F
:109A50007148B0F84002884229D16F48B0F84202FC
:109A6000884224D16C48B0F8440288421FD16A4829
:109A7000B0F8460288421AD16748B0F848028842D6
:109A800015D16548B0F84A02884210D16248B0F852
:109A90004C0288420BD16048B0F84E02884206D191
:109AA0005D48B0F85002884201D100F0F9FD4FF452
:109AB000F6725A495848F8F754FF574890F8000290
:109AC00057498873544890F801125548C173524859
:109AD00090F80212524801744F4890F8031250480F
:109AE00041744D4890F804024D4908704A4890F876
:109AF00005024870484890F806028870464890F879
:109B00000702C870444890F8081245484175424819
:109B100090F80912424881753F4890F80A0240497E
:109B200008713D4890F80B123D4841713A4890F851
:109B30000C123B488171384890F80D123848C171B9
:109B4000354890F80E0237498873334890F80F1261
:109B50003448C173304890F81012324801742E48CE
:109B600090F811122F4841742B4890F812022D4999
:109B70000870294890F813024870274890F814029A
:109B80008870254890F81502C870234890F816127E
:109B900024484175204890F81712224881751E48C4
:109BA00090F818021F4908711B4890F819121D48B7
:109BB0004171194890F81A121A488171164890F8A4
:109BC0001B121848C171144890F81C121548C17531
:109BD000114890F81D12134801760F4890F81E1294
:109BE000104841760C4890F81F120E4881760A48BA
:109BF00090F820120B48C176074890F821120948C6
:109C000001770020044981F8D8030846B0F8220201
:109C10000549088410BD0000E80A0020D40C00208B
:109C200048000020E80E0020581800202DE9F841D7
:109C300003460C4621461D46960802F00307002005
:109C400005E055F820C0C1F800C0091D401CB04215
:109C5000F7D36FB155F826000090EC46002004E0E1
:109C60001CF8008001F80080401CB842F8D300BF07
:109C7000BDE8F8812DE9FC5F0746884615460024BB
:109C80004646A808019005F00309BA46F9F7E4FE34
:109C90003846FFF7FFFD044624B1F9F77BFE204666
:109CA000BDE8FC9F4FF0000B0FE0D6F800C0624605
:109CB000002351460220F9F777FE044604B107E07D
:109CC0000AF1040A361D0BF1010B01988345ECD310
:109CD00000BFB4B9B9F1000F13D04FF0FF300090BE
:109CE000EB46002003E0315C0BF80010401C4845B7
:109CF000F9D3002351460220009AF9F755FE044695
:109D000000BFF9F747FE2046CAE7000010B5174824
:109D100090F8150850B14FF400511548FAF74CF877
:109D2000012291031248FAF751F809E04FF48041FB
:109D30000F48FAF741F8012251030D48FAF746F8A7
:109D40000C4890F8D80301280FD13220F9F756FAC1
:109D50004FF480410648FAF72FF83220F9F74EFA0F
:109D60004FF400510248FAF727F810BD081A0020F6
:109D700000100140E80A002010B5002409E032205C
:109D8000F9F73CFA4FF480410348FAF715F8601CE4
:109D9000C4B2142CF3DB10BD0010014070B50446B2
:109DA0000E46154600BFA07C0028FCD00020A07401
:109DB000A08BA84200DAA58B2A4631466069F8F7E5
:109DC000D0FD2A4661696068FBF7E2F970BD10B505
:109DD000044660680068C06840F010006168096867
:109DE000C860E28BA1696068FBF7BAF910BD70B575
:109DF00004466068FAF74EFEE08BE168096849683E
:109E0000401A86B206B970BD002506E0A269511954
:109E1000206802F09BFF681C85B2B542F6DB204645
:109E200000F040F8E28BA1696068FBF799F900BF88
:109E3000E9E7000070B50446A08C618C884226DA00
:109E4000206880892084204600F032F8208CE18B45
:109E500088421CDC208CD0B1208CB0F5007F03D967
:109E6000206802F027FF12E0002506E0084A511999
:109E7000206802F027FF681C85B2208CA842F5DC20
:109E8000E06B20B1218C22460148E36B984770BDFE
:109E9000B829002090F82620012A02D1428C0A44D9
:109EA00042847047012180F82610002141847047C8
:109EB000002180F82610418470472DE9F0410446C6
:109EC0000F461646A08B96FBF0F01FFA80F800258F
:109ED00007E0A28B02FB05712046FFF75FFF681CBD
:109EE00085B24545F5DBA08B00FB156086B20EB947
:109EF000BDE8F081A08B00FB057132462046FFF7DC
:109F00004DFF00BFF4E701218174704710B512497D
:109F100048688047FDF77CFFFDF7A4FFF9F774F967
:109F2000002415E040F2231161430C4A12681432F8
:109F300002EBC10000F00EFA002240F22310604351
:109F400006490968143101EBC0000274601CC4B2F8
:109F5000012CE7DB10BD0000A80A002088090020C2
:109F600010B5124948688047FDF766FFFDF7F2FF1C
:109F7000F9F7B2F9002415E040F2231161430C4ACD
:109F80001268143202EBC10000F002FA002240F223
:109F90002310604306490968143101EBC0000274C4
:109FA000601CC4B2012CE7DB10BD0000A80A002031
:109FB0002818002070B500BF1720FDF7ABF8064643
:109FC0000A20F9F77BFC0024D0E00120A0403040BB
:109FD00000287DD040F223116143694A126814328F
:109FE00012F831000221FDF7DDF8054640F2231199
:109FF0006143634A1268143212F831002A46022182
:10A00000FEF79CF905F00100A0B140F22310604377
:10A010005B490968143101EBC000007C40F002028A
:10A0200040F2231004FB00F155480068143000EBA7
:10A03000C100027405F00200F8B140F2231161433F
:10A040004F4A1268143212F8310010220121FEF733
:10A0500075F940F223116143494A1268143202EB48
:10A06000C10000F077F9002240F223106043444918
:10A070000968143101EBC000027405F0100098B1BA
:10A0800040F2231060433E490968143101EBC000DF
:10A09000407C40F0020240F22310604338490968D6
:10A0A000143101EBC000427405F00400A8B140F285
:10A0B0002310604332490968143101EBC000407C31
:10A0C00040F0010240F2231060432D49096800E08E
:10A0D00044E0143101EBC000427405F00800E8B31D
:10A0E00040F223116143264A1268143212F83100FB
:10A0F0002A460221FEF722F940F223116143204A49
:10A100001268143212F8310010220121FEF716F9FC
:10A110000A20F9F7D3FB40F223116143184A126871
:10A12000143202EBC10000F015F940F22311614333
:10A13000134A1268143202EBC10000F047F9002202
:10A1400040F2231060430E490968143101EBC0004E
:10A15000027440F223106043094900E004E00968FA
:10A16000143101EBC0004274601CC4B2012CFFF634
:10A170002CAF1720FCF7CEFF00B11DE770BD00002B
:10A180008809002070B500BF1720FCF7E7FF0646DE
:10A190000A20F9F793FB0024D0E00120A0403040D2
:10A1A00000287DD040F223116143694A12681432BD
:10A1B00012F831000221FDF71FF8054640F2231185
:10A1C0006143634A1268143212F831002A460221B0
:10A1D000FEF7D4F805F00100A0B140F2231060436F
:10A1E0005B490968143101EBC000007C40F00202B9
:10A1F00040F2231004FB00F155480068143000EBD6
:10A20000C100027405F00200F8B140F2231161436D
:10A210004F4A1268143212F8310010220121FEF761
:10A22000ADF840F223116143494A1268143202EB3F
:10A23000C10000F0ADF8002240F223106043444911
:10A240000968143101EBC000027405F0100098B1E8
:10A2500040F2231060433E490968143101EBC0000D
:10A26000407C40F0020240F2231060433849096804
:10A27000143101EBC000427405F00400A8B140F2B3
:10A280002310604332490968143101EBC000407C5F
:10A2900040F0010240F2231060432D49096800E0BC
:10A2A00044E0143101EBC000427405F00800E8B34B
:10A2B00040F223116143264A1268143212F8310029
:10A2C0002A460221FEF75AF840F223116143204A40
:10A2D0001268143212F8310010220121FEF74EF8F4
:10A2E0000A20F9F7EBFA40F223116143184A126889
:10A2F000143202EBC10000F04BF840F2231161432D
:10A30000134A1268143202EBC10000F092F80022E6
:10A3100040F2231060430E490968143101EBC0007C
:10A32000027440F223106043094900E004E0096828
:10A33000143101EBC0004274601CC4B2012CFFF662
:10A340002CAF1720FCF70AFF00B11DE770BD00001D
:10A350002818002010B50446207840F2B45212218B
:10A36000FEF72CF8A178637841EA032220780421D3
:10A37000FEF724F8237AE17943EA012220781021BC
:10A38000FEF71CF82078E21C0C21FEF757F810BDF0
:10A3900010B50446207840F2B4521221FEF72EF890
:10A3A000A178637841EA032220780421FEF726F899
:10A3B000237AE17943EA012220781021FEF71EF882
:10A3C0002078E21C0C21FEF765F810BD10B504469C
:10A3D000207C68BBE07B20B1012811D0022825D168
:10A3E00019E02078FDF79BF8FF2806D101202074A2
:10A3F0002078022103F062F801E00020207416E0CA
:10A400002078FDF746F8FF2802D10120207401E0F2
:10A41000002020740BE02078FDF7E7F8FF2802D138
:10A420000320207401E00020207400E000BF00BF82
:10A4300010BD10B50446207C68BBE07B20B101282C
:10A4400011D0022825D119E02078FDF79BF8FF28CC
:10A4500006D1012020742078022103F038F801E0B1
:10A460000020207416E02078FDF736F8FF2802D18E
:10A470000120207401E0002020740BE02078FDF71B
:10A48000D2F8FF2802D10320207401E000202074BC
:10A4900000E000BF00BF10BD70B500240BE040F22B
:10A4A00023116143364A1268143202EBC100FFF7F0
:10A4B0008DFF601CC4B2012CF1DBFFF77BFD002493
:10A4C0005BE040F2231060432D490968143101EB31
:10A4D000C000407C00F00100E8B340F2231060436C
:10A4E00027490968143101EBC000407C20F00102CB
:10A4F00040F22310604322490968143101EBC00087
:10A50000427440F2231060431D4A1268143202EB79
:10A51000C00000F112010020FCF7CAFC054640F221
:10A520002310604316490968143101EBC000D0F8CC
:10A530001409F8B140F223126243114E3668143602
:10A5400006EBC20202F1120140F2231262430C4EEA
:10A550003668143600E00EE006EBC20040F223122B
:10A560006243074E3668143606EBC202D2F814393D
:10A570002A46984700BF601CC4B2012CA1DB70BD05
:10A580008809002070B500240BE040F223116143DC
:10A59000394A1268143202EBC100FFF74AFF601C0F
:10A5A000C4B2012CF1DBFFF7EDFD002461E040F2C5
:10A5B0002310604330490968143101EBC000407C2E
:10A5C00000F00100002852D040F2231060432A49D5
:10A5D0000968143101EBC000407C20F0010240F218
:10A5E0002310604324490968143101EBC000427410
:10A5F00040F223126243204B1B68143303EBC20268
:10A6000002F1120140F2231262431B4B1B68143308
:10A6100013F83200FCF7E4FC054640F223106043D7
:10A6200015490968143101EBC000D0F81409E8B1EC
:10A6300040F223126243104E3668143606EBC20213
:10A6400002F1120140F2231262430B4E36681436B7
:10A6500006EBC20040F223126243074E36681436FE
:10A6600006EBC202D2F814392A46984700BF601C94
:10A67000C4B2012C9BDB70BD2818002010B5024825
:10A68000F9F7E1FB10BD00006C2200200348406890
:10A6900040F480700149486070470000002004E0E9
:10A6A00010B518216A48F8F775F918216848183864
:10A6B000F8F770F9182166487830F8F76BF9182127
:10A6C00063483038F8F766F9182161486030F8F7C8
:10A6D00061F918215E484830F8F75CF918215C48A8
:10A6E0001830F8F757F9182159483030F8F752F96F
:10A6F00045F24F315748A0F83E1245F25F31A0F8BD
:10A70000401244F25F11A0F8421244F24241A0F814
:10A71000441244F24451A0F8461243F23101A0F829
:10A72000481244F25F11A0F84A1243F25F31A0F8D8
:10A730004C1245F23101A0F84E1244F65321A0F814
:10A74000261245F25071A0F8281243F23151A0F8B8
:10A750002A1243F23001A0F82C1244F24421A0F84E
:10A760002E1243F22D61A0F8301243F23501A0F809
:10A77000321242F65351A0F8341243F23201A0F8DB
:10A7800036123821A0F8381244F25331A0F8CE1214
:10A7900045F25251A0F8D01244F24221A0F8D21250
:10A7A00045F24521A0F8D41244F24121A0F86E12DE
:10A7B00044F24341A0F8701243F24511A0F872121E
:10A7C0003121A0F8741244F24121A0F8861244F21B
:10A7D0004341A0F8881243F24511A0F88A123121B2
:10A7E000A0F88C1244F65321A0F89E1243F25601B1
:10A7F000A0F8B61242F63261A0F8B81243F2304126
:10A80000A0F8BA1243F22E01A0F8BC1242F6306151
:10A81000A0F8BE1243F23001A0F8C01243F25F016B
:10A82000A0F8C21242F63061A0F8C41243F23071AF
:10A83000A0F8C61245F25F61A0F8C81242F6346172
:10A84000A0F8CA123121A0F8CC12FFF747F810BDCA
:10A850003E0D0020E80A00207047000010B54FF4BC
:10A8600000710E48F9F7A0FA38B90D480068008861
:10A87000401C0B490968088003E00020084909686A
:10A880000880074800680088B0F5FA7F05DB0549B5
:10A89000D1F8E8038047F9F7AFFB10BD000C014089
:10A8A000E00E0020E80A00202DE9FE4F06460F4684
:10A8B00090469946DDE90CAB1AA207CA8DE807005D
:10A8C00000244FF4FA6507E0284600F097F800F2FC
:10A8D0006D100444681C85B2B542F5DB01250CE01F
:10A8E000681E1DF800000444022D04D1304600F01B
:10A8F00085F800B1641C681CC5B2BD42F0DBA8F14C
:10A90000010004440A486043C9EB4911C1EB092125
:10A9100000EB0110CAEB0A1100EB81005844BDE8BE
:10A92000FE8F00001F1C1F1E1F1E1F1F1E1F1E1F2D
:10A93000805101002DE9F04104460D461646374688
:10A940000FB104B10DB9BDE8F0812A462146384661
:10A95000FB6A984700BFF6E7FEB505460C4616466B
:10A9600037460FB105B104B9FEBD082C0DDB2246F8
:10A9700029466846FAF706FE012806D106483246FF
:10A980002146436928469847EEE72246294638463D
:10A99000FB6A984700BFE7E78818002070B50446B7
:10A9A0000D461646B4B1ADB1A6B10B48844207D1ED
:10A9B000143832462946D0F83C392046984709E0F9
:10A9C0000648844206D1143832462946D0F83C392C
:10A9D0002046984770BD00005C000020FC0E00205F
:10A9E00038B504460D46E0B200900348012269469E
:10A9F000C36A984738BD0000640A002001460A4631
:10AA0000C81701EB90708010A1EB800028B964207A
:10AA100091FBF0F300FB131030B94FF4C87091FBB9
:10AA2000F0F300FB131008B9012070470020FCE789
:10AA3000F9F71CFAFCF730FEFAF768FCFAF724FC89
:10AA4000FAF7F2FCFAF748FDFAF77EFDFAF760FD37
:10AA5000FAF7FEFCFAF71EFDF8F7ACFA04E0F8F797
:10AA600003FB0248F9F7EFF9F9E700006C22002038
:10AA700070B503460C4603E014F8015B03F8015B74
:10AA8000151EA2F10102F7D170BD000010B51449E6
:10AA90001448C0F828190020134909684881124950
:10AAA000096808701049096848600F490968087208
:10AAB0000D4909680873A8210B4800681430F7F79E
:10AAC00069FF4FF4EE6108480068C030F7F762FF95
:10AAD0000548006800F5006000210163416310BD76
:10AAE000EDAA0008E80E0020502200202DE9F047D2
:10AAF00081460C469046B8F1090F01DABDE8F087AF
:10AB00006078217840EA01268F4800684089B04289
:10AB100000D0F3E7A07808B9E07800B1EEE7A079BB
:10AB2000012800D0EAE7E079832804D10020864993
:10AB300009680870E2E7E07906280CD182480068CD
:10AB4000C089B04206D101207F49096808737E4957
:10AB500009680874D2E7E07986280DD17A48006840
:10AB6000C089B04207D103207749096808730020E3
:10AB7000754909680874C1E7E079032800D0BDE78A
:10AB8000257A05F10900404500DDB7E76E48006809
:10AB90000078012806D002282CD0032859D0042898
:10ABA0007ED182E0102D24D104F1090000210AE0B9
:10ABB0004278037842EA0323634A1268143222F887
:10ABC0001130801C491C0829F2DB02215E4A126800
:10ABD000117000215C4A126851605B4A1268117260
:10ABE000594A1268517400225749096881F815289A
:10ABF00000BFA6E0682D2BD104F10900002111E06F
:10AC000003781B06477843EA0743877843EA07231C
:10AC1000C77843EA07024C4B1B68243343F82120D2
:10AC2000001D491C1A29EBDB0321474A12681170E9
:10AC30000021454A12685160434A12681172424A23
:10AC40001268517400224049096881F8152800BF34
:10AC500077E0062D28D104F1090700200AE0797871
:10AC60003A7841EA0222384909688C3121F81020EB
:10AC7000BF1C401C0328F2DB04203349096808701C
:10AC8000F9F7AAF830490968486000202E49096898
:10AC900008722D490968487400212B48006800E0BB
:10ACA0004EE080F8151800BF4BE0142D47D104F199
:10ACB000090797F800A0BAF1140F00DDAA46BAF10F
:10ACC000000F0DDD5246791C1F480068A630F7F7CB
:10ACD00048FE00211C480068A63000F80A1004E075
:10ACE00000211948006880F8A61000200FE002211A
:10ACF00001EB4001795C012202EB4002BA5C41EABF
:10AD0000022211490968923121F81020401C0A28BA
:10AD1000EDDB00200C4909680870F9F75DF80A4975
:10AD200009684860002008490968087206490968EE
:10AD3000487400210448006880F8151800BF00BF5F
:10AD400000BF00BF00BFD9E6502200203EB5044638
:10AD50000D461B4800684089401C19490968488114
:10AD6000174800684089000A8DF800001448006800
:10AD7000807A8DF8010000208DF802008DF8030024
:10AD80008DF8040006208DF8050001208DF80600DE
:10AD900003208DF80700200A8DF80800E0B28DF836
:10ADA0000900280A8DF80A00E8B28DF80B00054862
:10ADB0000C226946D0F83C39143098473EBD00005B
:10ADC00050220020E80E00203EB504460D462248E1
:10ADD00000684089401C2049096848811E48006875
:10ADE00040891D490968C88102201B490968087308
:10ADF0000020194909680874174800684089000A4A
:10AE00008DF8000014480068807A8DF80100002059
:10AE10008DF802008DF803008DF8040006208DF8EF
:10AE2000050001208DF8060006208DF80700200A95
:10AE30008DF80800E0B28DF80900280A8DF80A00A4
:10AE4000E8B28DF80B0005480C226946D0F83C3971
:10AE5000143098473EBD000050220020E80E00202C
:10AE600070B5474890F8240000F0020048B900206F
:10AE700044490968087001214248006880F81518A3
:10AE800070BDF8F7A9FF04463E480068007878B91D
:10AE900008210020FFF75AFF01203A49096808708D
:10AEA0003848006844600020364909680872E7E7BE
:10AEB000344800684068201AB0F5FA7F5DD3314805
:10AEC0000068007A401C2F49096808722D48006804
:10AED000007A042821DA2B4800680078012806D07F
:10AEE000022807D0032808D004280CD108E0002548
:10AEF000082609E03225342606E0FA25032603E079
:10AF0000FD250A2600E0BBE700BF31462846FFF7D3
:10AF10001DFF1C48006844602FE0002019490968A3
:10AF2000087218480068407C401C1649096848743B
:10AF300014480068407C032805DB012111480068A3
:10AF400080F8151804E000210E48006880F81518F4
:10AF50000C4800680078042807DA0A48006800787E
:10AF6000401C08490968087003E000200549096889
:10AF70000870002003490968486000BF80E70000AE
:10AF8000E80E0020502200202DE9F04104460A4836
:10AF900090F8240000F0020008B9BDE8F0810748ED
:10AFA0000068478C782527EA0506264331460720A6
:10AFB000FFF70AFF00BFF0E7E80E00205022002054
:10AFC0000146080240EA212080B2704710B502F025
:10AFD00065FA04460548007828B9012C03D10449D4
:10AFE000D1F8300980470148047010BD44000020AA
:10AFF0004800002010B502F059FA044605480078D0
:10B0000028B9012C03D10449D1F8300980470148FF
:10B01000047010BDE40E0020E80E00202DE9F0477A
:10B0200005460E464FF00009376870791A282ED071
:10B0300011DC112822D007DCA0B308281CD0092875
:10B040001BD0102838D11EE0122821D018282CD06F
:10B05000192831D114E0282825D006DC1C281DD061
:10B06000202821D0242827D117E0292807D02A28F2
:10B070000CD02C2820D10FE000BF00BF00BF00BFC4
:10B0800096F807801BE096F8078018E000BF00BF25
:10B09000F0794FEA400812E000BF00BFF0794FEAB4
:10B0A00080080CE005E000BF00BFF0794FEAC0085F
:10B0B00005E04FF0010802E04FF0000800BF00BFBC
:10B0C000B8F1FF0F0BDC7079012101EB80002870D3
:10B0D00085F8018008F102001FFA80F90DE070790F
:10B0E000022101EB800028704FEA2820687085F863
:10B0F000028008F103001FFA80F970791A2859D0EC
:10B1000011DC112834D007DCF0B108282ED0092832
:10B110002DD0102840D140E012284CD018287DD0E6
:10B120001928F7D126E0282879D006DC1C2866D01B
:10B13000202875D02428EDD160E0292819D02A28AC
:10B1400037D02C28E6D158E0287800F003010129F7
:10B1500005D13068007868700220BDE8F0870020D3
:10B16000687030680078A8700320F6E700BF00BF61
:10B1700000BF00BF287800F0030000F1010AF07959
:10B18000012803D1387805F80A0005E0F27905EBCB
:10B190000A003946F7F7E5FB99E0287800F003004C
:10B1A00000F1010AF27905EB0A003946F7F7D9FBFD
:10B1B0008DE000BF00BF297801F00301481CF17940
:10B1C000012905D1797829543A78411C6A5413E051
:10B1D00000240EE0012101EB4401795C00EB440204
:10B1E000A95417F8142000EB4401491C6A54611C4F
:10B1F000CCB2F179A142EDDC69E000BF00BF297853
:10B2000001F00301481CF17901290FD1F978295483
:10B21000BA78411C6A547A78811C02E02DE02AE059
:10B220002AE06A543A78C11C6A5423E000241EE0E4
:10B23000032101EB8401795C00EB8402A954022113
:10B2400001EB84017A5C00EB8401491C6A54012102
:10B2500001EB84017A5C00EB8401891C6A5417F8C5
:10B26000242000EB8401C91C6A54611CCCB2F17922
:10B27000A142DDDC2BE000BF00BF287800F0030016
:10B28000411CF07901280BD1002406E0C4F107002D
:10B29000385C0A19A854601CC4B2082CF6DB15E00F
:10B2A000002410E000200AE0072202EBC402121A78
:10B2B000BA5C01EBC4030344EA54421CD0B2082830
:10B2C000F2DB601CC4B2F079A042EBDC00BF00BF2F
:10B2D000484642E770B504460D460021284602F074
:10B2E000BEF820600021281D02F09AF8A080A879FD
:10B2F000A071E879E071287A2072687A6072002182
:10B3000005F10A0002F0ABF8E06070BD02490348A5
:10B31000C0F8281970470000E1C900084800002063
:10B3200070B505460C460E2C00DA70BD294645481E
:10B330000068FFF7CFFF434800680068001DA04287
:10B3400000D0F2E73F480068007A00B1EDE73D48E1
:10B350000068407A0A2871D2DFE800F005213A3B04
:10B3600053546C6E706F37480068008C354909681B
:10B370008988884200D0D8E73248006831490E6891
:10B380004ECE10304EC0A4F10E0082B22E4805F110
:10B390000E0103692B480068103098474FE0294898
:10B3A000006828490B68D3E901621968DB68C0E9C5
:10B3B0000562C361016102212248006841760023D1
:10B3C0001A4619461F480068103000F051F836E060
:10B3D00035E01C4802680668D6E901313068F66835
:10B3E000C2E90616C2E90403042116480068417642
:10B3F00000231A46194613480068103000F038F848
:10B400001DE01CE00F4801680668D6E901033268B8
:10B41000F668C1E90636C1E904200621094800683A
:10B42000417600231A46194606480068103000F09D
:10B430001FF804E003E001E001E000E000BF00BF0E
:10B4400000BF72E7841800202C18002070B5044655
:10B450000D4629462046F7F7D0FE04482A462146E5
:10B46000D0F83C391430984770BD000048000020E7
:10B470002DE9F0470446884616469946184D06F1D0
:10B480000A00206000222946206801F0ACFFA08855
:10B490000022291D01F08AFFA079A871E079E871E6
:10B4A000207A2872607A6872002205F10A01E06849
:10B4B00001F099FF0E27B8F1000F07D036B1E81957
:10B4C00032464146F7F74DFAB81987B23946284651
:10B4D000FFF7BCFF39462846F7F78FFEBDE8F08737
:10B4E0002040002004480549C8630549C863054851
:10B4F0000549C86370470000915F0008DC0900201F
:10B50000200A002035A90008640A002070470000C6
:10B510002DE9F05F804689464FF0000A002700259C
:10B5200050E00AF1010000F0FF0ABAF1640F00DDFB
:10B530004AE018F80530991003F0030C681C85B236
:10B540000022BCF1010F04D118F80520681C85B257
:10B550000FE0BCF1020F09D1681C18F8000018F8C0
:10B5600005B040EA0B22A81C85B202E00020BDE82D
:10B57000F09F91B9814800EBC7004171DFF8FCB141
:10B580000BEBC70B8BF8062008EB0500DFF8ECB1DE
:10B590004BF83700781CC7B213E0784800EBC700BF
:10B5A0004171DFF8D8B10BEBC70B8BF8062008EB25
:10B5B0000500DFF8C8B14BF83700A81885B2781C31
:10B5C000C7B200BF4D45ACDB00BF00250024CFE073
:10B5D0006A4800EBC40040791A2847D010DC1128D3
:10B5E00021D006DC08281CD009281BD010287DD1CA
:10B5F0001CE012283BD0182879D01928F7D114E084
:10B60000282875D006DC1C2859D0202871D0242881
:10B61000EDD153E0292807D02A2826D02C28E6D1BE
:10B620004BE000BF00BF00BF00BF00BF534B03EBA8
:10B63000C4039A79514B53F83410514B5819F7F70A
:10B6400090F94E4800EBC40080794C4901EBC401ED
:10B65000C8714B482844494941F83400084600EB7A
:10B66000C4008079284485B27FE000BF00BF434911
:10B6700051F83400002607E0C6F10101415CAA1927
:10B680003F4B9954711CCEB2022EF5DB3B4A02EBC4
:10B69000C402917901EBD1725210384B03EBC40311
:10B6A000DA7137492944354A42F83410114601EB22
:10B6B000C401897929448DB257E000BF00BF2F48EB
:10B6C00050F83410002607E0C6F10300085CAA1900
:10B6D0002B4B9854701CC6B2042EF5DB274A02EBA4
:10B6E000C4029079C21700EB927203E03CE014E0D0
:10B6F00011E011E09210214B03EBC403DA712048F2
:10B7000028441E4A42F83400104600EBC4008079F9
:10B71000284485B229E000BF00BF184850F8341013
:10B72000002607E0C6F10700085CAA19144B9854DC
:10B73000701CC6B2082EF5DB104A02EBC4029079E9
:10B74000C21700EB5272D2100C4B03EBC403DA7138
:10B750000B482844094A42F83400104600EBC40064
:10B760008079284485B200E000BF00BF601CC4B2ED
:10B77000BC42FFF62DAF3846F9E60000B83B00208A
:10B78000483D00202DE9F04FB3B00546894692466A
:10B79000E879A97901F07F0140EA0127A879012120
:10B7A000B1EBD01F06D040F20C60874202D033B01C
:10B7B000BDE8F08F51464846FFF7AAFE064640F224
:10B7C0000110874205D040F20D10874201D006B922
:10B7D000EDE78E49E8680968086040F21F21781A91
:10B7E0008F427DD008DCA7F20110002879D0022812
:10B7F00009D00C2876D191E0122829D0A0F2ED30A2
:10B800000028F7D182E006B9D1E74FF00008002404
:10B8100013E07F4800EBC40040792C280BD17C4911
:10B8200051F8340041464A1C02F0FF0801AA03689F
:10B8300042F8213000BF601CC4B2B442E9DBB8F169
:10B84000000F04DD424601A9284600F051FDDAE070
:10B850006F48846923466FA20B2130A8FCF7A0FE35
:10B8600005226DA130A8F7F7D7F848B96C48D0F891
:10B87000401808208847012164480068417138E079
:10B88000042268A130A8F7F7C7F848B96448D0F88F
:10B8900040181020884702215C480068417128E068
:10B8A000092262A130A8F7F7B7F848B95C48D0F888
:10B8B000401820208847032154480068417118E04F
:10B8C0000A225DA130A8F7F7A7F860B95448D0F86C
:10B8D00040184020884704214C480068417108E026
:10B8E00022E00DE08EE000221146284600F060FEC6
:10B8F0005DE746480068016844480068816082E06E
:10B9000000221146284600F03DFC7CE0404840798A
:10B91000082802D13E49086800BF74E000221146A1
:10B92000284600F07BFC6EE039484079102868D149
:10B9300037480468A078303800EB80004FF4FA6193
:10B9400001EB4001E078303808441FFA80F8607954
:10B9500030382179303901EB810100EB410000F0F2
:10B96000FF0BE0793038A179303901EB810100EB30
:10B970004100C0B23290607A3038217A303901EB20
:10B98000810100EB4100C0B23190E07A3038A17AF9
:10B99000303901EB810100EB4100C0B23090607B97
:10B9A0003038217B303901EB810100EB4100C0B21E
:10B9B0002F9000202E90E07B3038A17B303901EBB6
:10B9C000810100EB41002E90DDE92F212E98CDE979
:10B9D000001202901B48D0F820C059464046DDE9CD
:10B9E0003132E04730B100231A461946284600F0AC
:10B9F000B7FD05E0012300221146284600F0B0FD06
:10BA000000BF00E000BF00BF00BFD0E64C18002020
:10BA1000B83B00202573000073746172740000004D
:10BA2000081A002073746F700000000069646C6570
:10BA30005F6F70656E00000069646C655F636C6FBA
:10BA400073650000C00A00202DE9F04104460D4650
:10BA500016460448002332462946876A2046B847DE
:10BA6000BDE8F081581800202DE9F04F97B0F74954
:10BA7000B1F8101888B24FF47A72F5490988FBF7CB
:10BA80007FF9012870D1F2480188F048C0F81018F9
:10BA9000007EEE494A8B0021090241EA126140EA28
:10BAA000022641EAE077E948818B0023C08B1A0423
:10BAB00042EA10424FEA004C08461946134640EA53
:10BAC0000C041943E148008C0143E048408C41EAF2
:10BAD00000456FF47C021540DC4901F5006103C9A3
:10BAE00080EA060881EA0709D84901F6080103C976
:10BAF00060406940CDE90C01D649C869804783465A
:10BB0000D4481121826907A89047D348008CADF82A
:10BB100010009DF8120020F07F00801D8DF81200AB
:10BB20009DF8120020F0800080308DF812000B206C
:10BB30008DF8130000208DF814008DF81500C3480F
:10BB4000808AC0F300200290029870B10221BF48A1
:10BB500080F8141800F50060C0C0BC4800F608006A
:10BB600030C017B0BDE8F08F89E10021B74880F8F8
:10BB7000141890F8151890F82D08814253D0B34846
:10BB800090F8150801281FD1B04890F82D08D8B9B1
:10BB9000AE48C0F818B807A900F61C00F6F733FF46
:10BBA000AE4800680068401CAC4909680860AB48B2
:10BBB000006800680690002007AB01225A2100901F
:10BBC00003A800F071FD29E0A04890F8150828BBF3
:10BBD0009E4890F82D08012820D19C48D0F81808DC
:10BBE000ABEB000A9D4800680068401C9B4909684F
:10BBF00008609A48006800680690994B01225A2113
:10BC000003A8CDF800A000F04FFD0F219448F6F7EF
:10BC1000C1FE00218D48C0F8181800BF8B4890F86D
:10BC2000151880F82D18002188EA010089EA010121
:10BC300008430FD10023DDE90C0158405940084367
:10BC400008D1824800F50060C0C0804800F60800B6
:10BC500030C086E74FF0000A78E05246012100200C
:10BC6000CDE90E0108460E99F6F75CFE00EA0800E1
:10BC700001EA0901002358405940084362D0524666
:10BC800001210020CDE9100108461099F6F74AFE7F
:10BC900030403940002358405940084323D0714870
:10BCA0000078401C6F4908700AEB0A126E49501860
:10BCB00007A9F6F7A8FE6C48603840F82AB0674834
:10BCC00000680068401C65490968086063480068AE
:10BCD00000680690002007AB01225146009003A89F
:10BCE00000F0E2FC2EE05F480078012804DB5D48AC
:10BCF0000078401E5B4908705B48603850F82A00A5
:10BD0000ABEB00000190554800680068401C5349A7
:10BD100009680860514800680068069001980AEBBD
:10BD20000A11009050480B180122514603A800F058
:10BD3000BBFC00210AEB0A124B488154603840F8E2
:10BD40002A1000BF0AF1010000F0FF0ABAF1180F33
:10BD500083DB4FF0000A68E0524601210020CDE964
:10BD6000120108461299F6F7DDFDDDE90C231040BB
:10BD70001940002358405940084352D052460121EF
:10BD80000020CDE9140108461499F6F7CBFD2040B8
:10BD9000294000235840594008431DD00AEB0A129D
:10BDA0003249501807A9F6F72EFE314840F82AB05C
:10BDB0002A4800680068401C28490968086027482C
:10BDC000006800680690002007AB024651460090CC
:10BDD00003A800F069FC24E0254850F82A00ABEBEA
:10BDE000000001901D4800680068401C1B4909685C
:10BDF00008601A4800680068069001980AEB0A116A
:10BE000000901A480B180022514603A800F04CFC81
:10BE100000210AEB0A1215488154154840F82A10EF
:10BE200000BF0AF1010000F0FF0ABAF1400F93DBF6
:10BE3000064800F50060C0C0044800F6080030C0A5
:10BE400008480078002815DD012014E0081A0020B9
:10BE50002C000020C00A0020581800204C18002098
:10BE600024220020541800202C1B0020C41D002078
:10BE7000C41C00200020034981F8C00000BF00BF9F
:10BE80006FE60000081A00207FB53D49B1F834186C
:10BE900088B24FF47A723B490988FAF771FF01289A
:10BEA0006DD1384801883648C0F834180324458CD1
:10BEB00090F8150808B104241EE0314890F81408E1
:10BEC000022801D1022417E02D4890F8C000012873
:10BED00001D1012410E02A48008B402101EA2020F2
:10BEE00008B1032408E02648008B022101EA202043
:10BEF00008B1002400E00324214880F8314890F87C
:10BF00003008A0422ED02048008CADF804009DF8E7
:10BF1000060020F07F00801D8DF806009DF80600C9
:10BF200020F0800080308DF806000B208DF807008F
:10BF300000208DF808008DF809001448006800689A
:10BF4000401C1249096808601048006800680390A6
:10BF5000002322461946684600F01AF8084880F87F
:10BF6000304800BF064890F8151890F82D08814217
:10BF700004D0034890F8151880F82D1800BF7FBD35
:10BF8000081A00202C000020581800204C1800200F
:10BF90002DE9F04F8FB006468B461746744D0024AE
:10BFA00000200C900D90142107A8F6F7F3FC002058
:10BFB0008DF8050003200E900EA8009001208DF84A
:10BFC000070028196946FFF729F8204484B22C207D
:10BFD0008DF805004FF00108CDF8008001208DF8A4
:10BFE000070028196946FFF719F8204484B22C206D
:10BFF0008DF805004FF00209CDF8009001208DF872
:10C00000070028196946FFF709F8204484B2002088
:10C010008DF8050001200E900EA8009001208DF8EB
:10C02000070028196946FEF7F9FF204484B2002072
:10C030008DF8050002200E900EA8009001208DF8CA
:10C04000070028196946FEF7E9FF204484B22C2036
:10C050008DF805004FF0030ACDF800A001208DF8FF
:10C06000070028196946FEF7D9FF204484B2002052
:10C070008DF8050006200E900EA8009001208DF886
:10C08000070028196946FEF7C9FF204484B2102032
:10C090008DF8050037480090F6F793FCC0B28DF894
:10C0A000070028196946FEF7B9FF204484B2102022
:10C0B0008DF805002F4818300090F6F782FCC0B2CA
:10C0C0008DF8070028196946FEF7A8FF204484B2BE
:10C0D00010208DF80500274860300090F6F771FCBD
:10C0E000C0B28DF8070028196946FEF797FF204473
:10C0F00084B23A4620A10CA8FCF76AFA10208DF809
:10C1000005000CA8009001208DF807002819694649
:10C11000FEF784FF204484B218481121826902A8E6
:10C12000904710208DF8050002A80090F6F749FC12
:10C13000C0B28DF8070028196946FEF76FFF20444A
:10C1400084B210208DF805000DA0009003208DF81A
:10C15000070028196946FEF761FF204484B2224691
:10C1600029463046FFF770FC0FB0BDE8F08F0000A5
:10C17000B8330020560D002025640000C00A0020BE
:10C18000414C4C002DE9FE4305460F469046214E9A
:10C19000002400200290E879401CE871A87920F082
:10C1A0008000A87100208DF805000220029002A8EE
:10C1B000009001208DF8070030196946FEF72EFF28
:10C1C0002044C4B210208DF8050013480090F6F703
:10C1D000F8FBC0B28DF8070030196946FEF71EFF64
:10C1E0002044C4B210208DF805000B481838009088
:10C1F000F6F7E7FBC0B28DF8070030196946FEF785
:10C200000DFF2044C4B2224631462846FFF71CFCED
:10C21000BDE8FE83B8330020B60D00202DE9FF41B4
:10C2200006460F469046304D0024F079401CF071D0
:10C23000B07920F08000B07100208DF80900022054
:10C24000039003A8019001208DF80B00281901A983
:10C25000FEF7E4FE2044C4B20020009008208DF8D0
:10C260000900CDF804D001208DF80B00281901A990
:10C27000FEF7D4FE2044C4B200208DF8090002204D
:10C28000039003A8019001208DF80B00281901A943
:10C29000FEF7C4FE2044C4B210208DF809001348F4
:10C2A0000190F6F78EFBC0B28DF80B00281901A99A
:10C2B000FEF7B4FE2044C4B210208DF809000B48EC
:10C2C00018300190F6F77DFBC0B28DF80B002819ED
:10C2D00001A9FEF7A3FE2044C4B2224629463046F7
:10C2E000FFF7B2FBBDE8FF81B8330020860D0020C8
:10C2F0002DE9F04F87B0804689469246954E00243E
:10C3000098F80700401C88F8070098F8060020F00D
:10C31000800088F8060000200390002508E059F806
:10C320002500401C10B90120039003E0681CC5B231
:10C330005545F4DB00BF4FF0000B039810B14FF0F0
:10C340001F0B25E0002521E059F8250049F6724130
:10C35000884206D349F6A441884202D800F0010180
:10C3600071B149F63A51884202D3891C884207D9F3
:10C3700042F23751884203D040F6B931884203D1A6
:10C380000BF1010101F0FF0B681CC5B25545DBDB69
:10C3900000208DF81900CDF810B004A805900120F8
:10C3A0008DF81B00301905A9FEF738FE204484B231
:10C3B0000398002847D0002515E0674850F825006D
:10C3C000029000BF24208DF8190002A805900120DA
:10C3D0008DF81B00301905A9FEF720FE204484B219
:10C3E00000BF681CC5B21A2DE7DB002516E05A48CD
:10C3F000683030F81500029000BF2A208DF819002F
:10C4000002A8059001208DF81B00301905A9FEF740
:10C4100005FE204484B200BF681CC5B2032DE6DBD4
:10C4200000BF10208DF819004B4882300590F6F7B8
:10C43000C8FAC0B28DF81B00301905A9FEF7EEFD51
:10C44000204484B27EE000257AE059F8257042F25B
:10C450003750874212D100BF10208DF819003E4896
:10C4600082300590F6F7ADFAC0B28DF81B00301996
:10C4700005A9FEF7D3FD204484B25FE049F672407F
:10C48000874225D349F6A440874221D807F001000E
:10C49000F0B907F5C770C0F34700029002981A2858
:10C4A00015DA2D48029950F82100019000BF242090
:10C4B0008DF8190001A8059001208DF81B00301996
:10C4C00005A9FEF7ABFD204484B200BF00BF35E0F4
:10C4D00049F63A5087421DD3801C87421AD807F18B
:10C4E000C600C0B202901C486830029930F81100B2
:10C4F000019000BF2A208DF8190001A805900120A5
:10C500008DF81B00301905A9FEF788FD204484B280
:10C5100000BF13E040F6B93087420FD100BF2A2098
:10C520008DF819000D48059001208DF81B00301979
:10C5300005A9FEF773FD204484B200BF681CC5B294
:10C54000554582DB224631464046FFF77DFA07B06B
:10C55000BDE8F08FB83300202C1A002039220020CB
:10C560002DE9FF4182B004460F4690460F4E00254C
:10C57000E079401CE071A07920F08000A0710820D3
:10C580008DF8050005A8009001208DF807007019AE
:10C590006946FEF743FD2844C5B22A463146204687
:10C5A000FFF752FA06B0BDE8F0810000B833002072
:10C5B0002DE9F04186B006460F46904600200590D2
:10C5C0000490384D0024F8B20390F079401CF071CB
:10C5D000B07920F08000B07100208DF809000220B1
:10C5E000059005A8019001208DF80B00281901A9DC
:10C5F000FEF714FD2044C4B208208DF8090003A8FA
:10C60000019001208DF80B00281901A9FEF706FD05
:10C610002044C4B200208DF809000120059005A82F
:10C62000019001208DF80B00281901A9FEF7F6FCF6
:10C630002044C4B200208DF809000220059005A80E
:10C64000019001208DF80B00281901A9FEF7E6FCE6
:10C650002044C4B210208DF8090004A80190F6F718
:10C66000B0F9C0B28DF80B00281901A9FEF7D6FC6D
:10C670002044C4B210208DF8090004A80190F6F7F8
:10C68000A0F9C0B28DF80B00281901A9FEF7C6FC6D
:10C690002044C4B2224629463046FFF7D5F906B0F9
:10C6A000BDE8F081B83300202DE9F04393B0054692
:10C6B0000E4617469846DDF868905D4C00201290B3
:10C6C00010905C480F9095E80F00CDE90B23CDE961
:10C6D00009019DF82A0020F0800080308DF82A00A2
:10C6E00000208DF839000320119011A80D90012031
:10C6F0008DF83B00BDF8481060180DA9FEF78EFCC0
:10C70000BDF84810084480B212902C208DF83900F2
:10C7100010A80D9001208DF83B00BDF8481060185E
:10C720000DA9FEF77BFCBDF84810084480B21290BA
:10C730002C208DF839000FA80D9001208DF83B00BA
:10C74000BDF8481060180DA9FEF768FCBDF8481048
:10C75000084480B2129000208DF839000120119019
:10C7600011A80D9001208DF83B00BDF8481060180D
:10C770000DA9FEF753FCBDF84810084480B2129092
:10C7800000208DF839000220119011A80D90012091
:10C790008DF83B00BDF8481060180DA9FEF73EFC6F
:10C7A000BDF84810084480B212902C208DF8390052
:10C7B0002148089008A80D9001208DF83B00BDF895
:10C7C000481060180DA9FEF729FCBDF84810084470
:10C7D00080B2129000208DF839000120119011A82C
:10C7E0000D9001208DF83B00BDF8481060180DA990
:10C7F000FEF714FCBDF84810084480B212904B4676
:10C800000EA2142103A8FBF7CBFE03A8334612AAFD
:10C810002146CDE9007802900DA800F02DFBBDF86F
:10C820004820214609A8FFF70FF913B0BDE8F083AF
:10C83000B8330020FDB10100AC892300257500004C
:10C8400000B589B0634890F8150801282ED16248D8
:10C850000068407950B36148008CADF808009DF83D
:10C860000A0020F07F00801C8DF80A009DF80A0065
:10C8700020F0800080308DF80A0031208DF80B0008
:10C8800000208DF80C008DF80D005348006880687A
:10C8900004900022012101A8FFF78AFE00214E48E2
:10C8A0000068417100204B49087400BF4948007B73
:10C8B000022802D04748007B08B909B000BD4748AC
:10C8C000008CADF818009DF81A0020F07F00801C45
:10C8D0008DF81A009DF81A0020F0800080308DF845
:10C8E0001A0031208DF81B0000208DF81C008DF8F7
:10C8F0001D0039480068806808903648007C01288F
:10C9000011D135480068407901280CD10022114628
:10C9100005A8FFF74DFE00212F4800684171002057
:10C920002C49087454E02B48007C012811D12A4876
:10C930000068407902280CD10022114605A8FFF7B3
:10C9400037FE002124480068417100202149087405
:10C950003EE02048007C012811D11F480068407942
:10C9600003280CD10022114605A8FFF721FE002163
:10C9700019480068417100201649087428E01548DC
:10C98000007C012811D114480068407904280CD19A
:10C990000022114605A8FFF70BFE00210E48006893
:10C9A000417100200B49087412E00A48007C78B9F4
:10C9B00009480068407958B10022012105A8FFF715
:10C9C000F7FD002104480068417100200149087406
:10C9D00000BF72E7081A00204C18002058180020E9
:10C9E00070B506460C46154629462046FEF798FCCB
:10C9F00070BD00002DE9F04FF3B000207290A849FF
:10CA0000098888B241F28832A6490988FAF7B8F94C
:10CA100001287DD1A44890F8D8030228F9D1A14873
:10CA200000889F490860A149D1F88800F6F703F80B
:10CA300004460D469D49D1F88400F5F7FCFF0646F3
:10CA40000F469A49D1F88000F5F7F5FF80468946F0
:10CA50009649C86FF5F7EFFF82468B469349886F7A
:10CA6000F5F7E9FF719170909049486FF5F7E3FF92
:10CA70006F916E908D49086FF5F7DDFF6D916C90A9
:10CA80008A49C86EF5F7D7FF6B916A908749886E1F
:10CA9000F5F7D1FF699168908449486EF5F7CBFFAF
:10CAA000679166908149086EF5F7C5FF65916490BE
:10CAB0007E49C86DF5F7BFFF639162907B49886D31
:10CAC000F5F7B9FF619160907849486DF5F7B3FFCC
:10CAD0005F915E907549086DF5F7ADFF5D915C90D3
:10CAE0007249C86CF5F7A7FF5B915A906F49886C43
:10CAF000F5F7A1FF599158906C49486CF5F79BFFE9
:10CB0000579156906949086CF5F795FF559100E0EB
:10CB1000C3E054906549C86BF5F78DFF539152906F
:10CB20006249886BF5F787FF519150905F49486BD8
:10CB3000F5F781FF4F914E905C49086BF5F77BFF4D
:10CB40004D914C905949C86AF5F775FF4B914A9041
:10CB50005649886AF5F76FFF499148905349486AEA
:10CB6000F5F769FF479146905048B0F89010B0F83B
:10CB70008E004E4AB2F88C20CDE93AABCDE93C8923
:10CB8000CDE93E674195409442924491439071991A
:10CB90007098CDE938016F996E98CDE936016D999D
:10CBA0006C98CDE934016B996A98CDE932016999A5
:10CBB0006898CDE9300167996698CDE92E016599AD
:10CBC0006498CDE92C0163996298CDE92A016199B5
:10CBD0006098CDE928015F995E98CDE926015D99BD
:10CBE0005C98CDE924015B995A98CDE922015999C5
:10CBF0005898CDE9200157995698CDE91E015599CD
:10CC00005498CDE91C0153995298CDE91A015199D4
:10CC10005098CDE918014F994E98CDE916014D99DC
:10CC20004C98CDE914014B994A98CDE912014999E4
:10CC30004898CDE9100147994698CDE90E011B4867
:10CC4000408C1A49498C194A128C184B1B8CCDE91F
:10CC50000932CDE90B101548C08B1449C98B134A12
:10CC6000928B124B9B8BCDE90532CDE907100F4813
:10CC7000408B0E49498B0D4A128B0C4B1B8BCDE917
:10CC80000132CDE903100948C08A00900748C38AE1
:10CC9000828A818A0648FBF773FC73B0BDE8F08F87
:10CCA000B40A00202C000020E80A0020081A002006
:10CCB00024D5000800B97047002141610161C160BD
:10CCC00000BFF8E770B504460D460CB9002070BDF2
:10CCD000E06808B90020FAE745B1D4E90006236905
:10CCE00003FB060132462846FDF7C2FE2069401CC0
:10CCF000A16890FBF1F201FB12002061E068401E88
:10CD0000E0600120E3E770B504460D460CB9002051
:10CD100070BDD4E90210884201D10020F8E745B186
:10CD2000D4E90016636903FB061032462946FDF775
:10CD30009FFE6069401CA16890FBF1F201FB1200AC
:10CD40006061E068401CE0600120E1E770B50446E6
:10CD50000D460CB9002070BDD4E90210884204DAF7
:10CD600029462046FFF7CFFFF5E745B1D4E9001685
:10CD7000636903FB061032462946FDF779FE6069B8
:10CD8000401CA16890FBF1F201FB12006061206978
:10CD9000401CA16890FBF1F201FB12002061012010
:10CDA000D9E700002DE9FF5F0646894692469B467B
:10CDB0002D48B6FBF0F5B6FBF0F100FB11674FF420
:10CDC000FA6810E04046FDF719FE00F26D10009081
:10CDD0000098854200D207E000982D1A08F1010062
:10CDE0001FFA80F800BFEDE700BFA9F800801FA27E
:10CDF00007CA01AB07C34046FDF700FE10B11D2076
:10CE00008DF8050001240BE0601E01A9085CA84212
:10CE100000D907E0601E01A9085C2D1A601CC4B28D
:10CE20000C2CF1DD00BF8AF80040681C8BF8000074
:10CE30004FF46160B7FBF0F0C1B20E9801704FF48F
:10CE40006160B7FBF0F100FB11703C21B0FBF1F029
:10CE5000C1B20F9801703C20B7FBF0F100FB1171DB
:10CE600010980170BDE8FF9F805101001F1C1F1E1C
:10CE70001F1E1F1F1E1F1E1F2DE9F04FADB00446C1
:10CE80000E4615461F46DDE9379ADDF8D8800020AA
:10CE900025900320249001202390DAA0006822909E
:10CEA0001822D9A11CA8F5F75CFDDDA103C9CDE9C5
:10CEB0001A01DD4903C9CDE91801DB49083103C96D
:10CEC000CDE916011422D9A111A8F5F74AFDDCA27B
:10CED00007CA0EAB07C32822DCA104A8F5F741FD61
:10CEE0005A2F10D1B8F1010F0DD15A202B90E1A388
:10CEF000E5A22821E548FBF753FB1422E4A126A86C
:10CF0000F5F753FD2EE0B8F1000F14D02B97182F32
:10CF100003DAE24850F8270000E0E1A083465B46D0
:10CF2000D9A22821D948FBF73BFB1422D8A126A877
:10CF3000F5F73BFD16E007F118002B90412F03DABF
:10CF4000DB4850F8270000E0DAA083465B46CEA21B
:10CF50002821CE48FBF724FB1422DAA126A8F5F7F6
:10CF600024FD00BF0020607113202C902CA82060AD
:10CF70000120E071298888192146FEF74FF8298899
:10CF8000084428802C2060712BA820600120E071CB
:10CF9000298888192146FEF741F829880844288005
:10CFA0001020607126A82060F5F70BFDE07129883C
:10CFB00088192146FEF732F8298808442880102075
:10CFC0006071C4482060F5F7FCFCE071298888197D
:10CFD0002146FEF723F8298808442880BE48817D31
:10CFE000407D41EA0020BC49497CBB4A127CCDE926
:10CFF00000210290B848C37B827BB8A1BB48FBF7F5
:10D00000E7FA102060711CA82060F5F7DAFCE071E7
:10D01000298888192146FEF701F8298808442880C4
:10D0200010206071AB4818382060F5F7CAFCE07139
:10D03000298888192146FDF7F1FF298808442880AE
:10D040001020607191482060F5F7BBFCE0712988E1
:10D0500088192146FDF7E2FF29880844288010201E
:10D06000607111A82060F5F7ACFCE071298888197F
:10D070002146FDF7D3FF29880844288010206071DD
:10D080000EA82060F5F79DFCE071298888192146DB
:10D09000FDF7C4FF2988084428801020607194A1FE
:10D0A0005046F5F795FC28B91AA82060F5F789FCD9
:10D0B000E07104E018A82060F5F783FCE07129888E
:10D0C00088192146FDF7AAFF2988084428801020E6
:10D0D000607104A82060F5F774FCE0712988881954
:10D0E0002146FDF79BFF29880844288010206071A5
:10D0F000784890302060F5F764FCE0712988881941
:10D100002146FDF78BFF2988084428802C20607178
:10D110002BA820600120E071298888192146FDF79D
:10D120007DFF2988084428802C20607124A8206075
:10D130000120E071298888192146FDF76FFF2988B1
:10D14000084428802C20607123A820600120E07111
:10D15000298888192146FDF761FF2988084428801D
:10D1600010206071C4F800904846F5F72AFCE07181
:10D17000298888192146FDF751FF2988084428800D
:10D1800010206071C4F800A05046F5F71AFCE07159
:10D19000298888192146FDF741FF298808442880FD
:10D1A0001020607122A820600120E0712988881970
:10D1B0002146FDF733FF298808442880102060713C
:10D1C000444830302060F5F7FCFBE071298888196D
:10D1D0002146FDF723FF298808442880102060712C
:10D1E0003C4848302060F5F7ECFBE071298888194D
:10D1F0002146FDF713FF2988084428802DB0BDE89B
:10D20000F08F0000310000004944535F3136343064
:10D21000335F414C4552545F3631343131000000A8
:10D22000426567696E0000000CD500084F76657294
:10D230002054726967676572284869676829000029
:10D2400045717569706D656E740000007B653935D8
:10D2500037653331642D336534362D346136362DE0
:10D26000613661622D313434633062373164343079
:10D27000307D00005343525542424552204F66666E
:10D280006C696E650000000025730000D83F002027
:10D290004D616A6F7220416C61726D00A8180020A8
:10D2A000556E6B6E6F776E20416C61726D00000081
:10D2B00008190020556E6B6E6F776E205761726E85
:10D2C000696E67004D616A6F72205761726E696E98
:10D2D00067000000260D00204800002025642E2550
:10D2E000642E25642E25643A256400000040002049
:10D2F00030000000022800D17047012824D12049C5
:10D30000097809BB1F49C96B1F4A11601F49C96BC6
:10D310001F4A11601F49D1F828191F4A11601F497F
:10D32000D1F828191E4A11601E49164AD163174ABE
:10D33000D1631D4A1749C1F828291849C1F828297D
:10D3400001210F4A117019E0C0B90D49097801296E
:10D3500014D10D4909680B4AD1630D4909680B4A7C
:10D36000D1630D490A680B49C1F828290C490A689C
:10D370000A49C1F828290021014A117000BFBBE702
:10D3800064220020DC09002054220020640A0020CE
:10D3900058220020480000205C220020E80E0020D7
:10D3A0006022002059A900089DA9000810B5034675
:10D3B00062B9002007E0C0F10104E40043FA04F47C
:10D3C0000C54441CE0B20228F5DB0BE0012A09D121
:10D3D000002005E0C40043FA04F40C54441CE0B2FD
:10D3E0000228F7DB10BD10B5034662B9002007E044
:10D3F000C0F10304E40023FA04F40C54441CE0B22A
:10D400000428F5DB0BE0012A09D1002005E0C40067
:10D4100023FA04F40C54441CE0B20428F7DB10BDDA
:10D4200030B50246002361B9002007E0145CC0F16A
:10D430000105ED00AC402343441CE0B20228F5DBBB
:10D440000BE0012909D1002005E0145CC500AC40C7
:10D450002343441CE0B20228F7DB98B230BD30B55C
:10D460000246002361B9002007E0145CC0F1030507
:10D47000ED00AC402343441CE0B20428F5DB0BE094
:10D48000012909D1002005E0145CC500AC4023430C
:10D49000441CE0B20428F7DB184630BD10B52E203E
:10D4A000F9F738FE044604F0010010BD10B52E2037
:10D4B000F9F754FE044604F0010010BD70B50546AE
:10D4C0000C4622462F212846FAF738FF70BD70B56A
:10D4D00005460C4622462F212846FAF74FFF70BD1D
:10D4E00002030405060708090A0B0C0D0E0F1010A5
:10D4F0000102000000000000000001020304060712
:10D50000080900000000010203040000456E6400E9
:10D510000000000050554D500000000056322E32E1
:10D52000000000000D0A3D3D3D3D3D3D3D3D3D3D82
:10D53000204D6F64627573205443502044617461C0
:10D54000203D3D3D3D3D3D3D3D3D3D0D0A343030AE
:10D5500030307E34303030373A203078253034580F
:10D56000282575292C203078253034582825752910
:10D570002C20307825303458282575292C203078F7
:10D5800025303458282575292C20307825303458FA
:10D59000282575292C2030782530345828257529E0
:10D5A0002C20307825303458282575292C203078C7
:10D5B00025303458282575290D0A34303035307E11
:10D5C00034303130303A20252E33662C20252E334E
:10D5D000662C20252E33662C20252E33662C202504
:10D5E0002E33662C20252E33662C20252E33662CD8
:10D5F00020252E33662C20252E33662C20252E3315
:10D60000662C20252E33662C20252E33662C2025D3
:10D610002E33662C20252E33662C20252E33662CA7
:10D6200020252E33662C20252E33662C20252E33E4
:10D63000662C20252E33662C20252E33662C2025A3
:10D640002E33662C20252E33662C20252E33662C77
:10D6500020252E33662C20252E33662C20252E33B4
:10D66000660D0A34303235307E34303235333A206C
:10D6700025752C2025752C2025752C0D0A3D3D3D4A
:10D680003D3D3D3D3D3D3D20456E64206F6620445F
:10D69000756D70203D3D3D3D3D3D3D3D3D3D0D0A9F
:10D6A0000000000048482057617465722054616E84
:10D6B0006B2054656D702E0048482052656163747C
:10D6C000696F6E204368616D6265722054656D708C
:10D6D0002E00000048482045786875617374205416
:10D6E000656D702E000000004820436162696E6520
:10D6F0007420657868756173742054656D702E00B0
:10D70000482077617465722074616E6B2074656D5A
:10D71000702E000048207265616374696F6E20632B
:10D7200068616D6265722074656D702E0000000086
:10D730004C207265616374696F6E206368616D620D
:10D7400065722074656D702E00000000496E6C6576
:10D75000745F3120482062656C74206A61636B6578
:10D76000742074656D702E00496E6C65745F322094
:10D77000482062656C74206A61636B65742074650F
:10D780006D702E00496E6C65745F332048206265B1
:10D790006C74206A61636B65742074656D702E0013
:10D7A000496E6C65745F3420482062656C74206A31
:10D7B00061636B65742074656D702E00496E6C65D5
:10D7C000745F3520482062656C74206A61636B6504
:10D7D000742074656D702E00496E6C65745F362020
:10D7E000482062656C74206A61636B65742074659F
:10D7F0006D702E00482065786875617374207465BB
:10D800006D702E004F33204848000000454D4F00FA
:10D810005761746572204C65616B6167650000003B
:10D82000436F6E7461696E6D656E74204C65616BDB
:10D83000616765004820746F72636820566F6C746E
:10D84000616765004C20746F72636820566F6C745A
:10D8500061676500536D6F6B65000000486561741A
:10D8600020536F75726365204661696C757265003F
:10D87000484820496E6C6574312050726573737529
:10D88000726500004820496E6C65743120507265E5
:10D890007373757265000000484820496E6C6574AA
:10D8A0003220507265737375726500004820496EAE
:10D8B0006C65743220507265737375726500000078
:10D8C000484820496E6C65743320507265737375D7
:10D8D000726500004820496E6C6574332050726593
:10D8E0007373757265000000484820496E6C65745A
:10D8F0003420507265737375726500004820496E5C
:10D900006C65743420507265737375726500000025
:10D91000484820496E6C6574352050726573737584
:10D92000726500004820496E6C6574352050726540
:10D930007373757265000000484820496E6C657409
:10D940003620507265737375726500004820496E09
:10D950006C657436205072657373757265000000D3
:10D9600048204F75746C65742050726573737572BE
:10D97000650000004C2047656E6572616C2045783B
:10D9800068617573742050726573737572650000F9
:10D990004C2043444120207072657373757265009A
:10D9A0004C204E32207072657373757265000000F2
:10D9B000496E6C65742056616C76655F3120436CEE
:10D9C0006F7365204C696D6974205761726E696E62
:10D9D00067000000496E6C65742056616C76655F67
:10D9E0003220436C6F7365204C696D6974205761F8
:10D9F000726E696E67000000496E6C657420566136
:10DA00006C76655F3320436C6F7365204C696D697C
:10DA100074205761726E696E67000000496E6C6514
:10DA2000742056616C76655F3420436C6F7365209B
:10DA30004C696D6974205761726E696E67000000F1
:10DA4000496E6C65742056616C76655F3520436C59
:10DA50006F7365204C696D6974205761726E696ED1
:10DA600067000000496E6C65742056616C76655FD6
:10DA70003620436C6F7365204C696D697420576163
:10DA8000726E696E67000000496E6C6574205661A5
:10DA90006C76655F31204F70656E204C696D6974DE
:10DAA000205761726E696E6700000000496E6C65F8
:10DAB000742056616C76655F32204F70656E204C25
:10DAC000696D6974205761726E696E6700000000AD
:10DAD000496E6C65742056616C76655F33204F70BB
:10DAE000656E204C696D6974205761726E696E674E
:10DAF00000000000496E6C65742056616C76655FAD
:10DB000034204F70656E204C696D697420576172C6
:10DB10006E696E6700000000496E6C657420566186
:10DB20006C76655F35204F70656E204C696D697449
:10DB3000205761726E696E6700000000496E6C6567
:10DB4000742056616C76655F36204F70656E204C90
:10DB5000696D6974205761726E696E67000000001C
:10DB60005761726E696E67004848204C697175692B
:10DB700064204C6576656C004C4C204C697175696D
:10DB800064204C6576656C00447261696E20507546
:10DB90006D7020416C61726D00000000436972631A
:10DBA000756C6174696F6E2050756D7020416C6189
:10DBB000726D0000416C61726D000000436162692A
:10DBC0006E657420657868756173742054656D7036
:10DBD0002E2042726F6B656E000000005761746505
:10DBE000722074616E6B2074656D702E2042726FAE
:10DBF0006B656E005265616374696F6E2063686166
:10DC00006D6265722074656D702E2042726F6B6557
:10DC10006E000000457868756173742074656D70DE
:10DC20002E2042726F6B656E00000000496E6C65BD
:10DC300074312050726573737572652042726F6B18
:10DC4000656E0000496E6C657432205072657373A6
:10DC50007572652042726F6B656E0000496E6C656F
:10DC600074332050726573737572652042726F6BE6
:10DC7000656E0000496E6C65743420507265737374
:10DC80007572652042726F6B656E0000496E6C653F
:10DC900074352050726573737572652042726F6BB4
:10DCA000656E0000496E6C65743620507265737342
:10DCB0007572652042726F6B656E00004F75746CF3
:10DCC00065742050726573737572652042726F6B54
:10DCD000656E0000436162696E65742065786875E1
:10DCE0006173742070726573737572652042726F10
:10DCF0006B656E00546F72636820766F6C74616739
:10DD0000652073656E736F722042726F6B656E0073
:10DD1000546F7263682063757272656E74207365E8
:10DD20006E736F722042726F6B656E004361626941
:10DD30006E657420646F6F72206F70656E000000F6
:10DD40004820746F7263682043757272656E740048
:10DD50004C20746F7263682043757272656E740034
:10DD60005265616374696F6E204368616D626572AC
:10DD70002054656D702E4F75740000004C4C20507F
:10DD8000435720466C6F77004C2050435720666CF9
:10DD90006F7700004C204C535720666C6F77000063
:10DDA0005043572076616C766520636C6F736564B1
:10DDB000207769746820666C6F7700004C53572099
:10DDC00076616C766520636C6F7365642077697427
:10DDD0006820666C6F7700004820636174686F6428
:10DDE00065206E6974726F67656E20666C6F770070
:10DDF0004C20636174686F6465206E6974726F672C
:10DE0000656E20666C6F77004820526561637469A7
:10DE10006F6E204368616D6265722054656D702E6F
:10DE20002044656C61790000000000004CDE0008B1
:10DE3000000000206C2200005E2F00081CE100089A
:10DE40006C220020C42700004086000841321042A6
:10DE50000113127A131CD500162008534543533280
:10DE60002056322E322D56312E3030372E534A1056
:10DE700008C0A80101FFFFFF150C29AB7C1A010E99
:10DE8000326503FF138801FF01FF01FF01FF01FF5E
:10DE900001FF01FF01FF011E13B59F1B080D0413B5
:10DEA00099A41408CDAF140849802308481C207990
:10DEB0009D18190413B8254320013905A10B15B885
:10DEC00026185A2718E20213940914202823142034
:10DED000442412202904193913B82B1C20B82C0C07
:10DEE0004A0146320A1ACF7413BB9E1B0807941AC4
:10DEF000EF0C1A950C411A35081AAC441A70441AE2
:10DF0000CC406A88441A2D440A282E441AC4441A64
:10DF1000B8441A54D81A100439441A2F141A310C60
:10DF20004A02B6091E44138DA61B087D042BA80ABD
:10DF300040011213718F1408E190140839921408EB
:10DF400055931B08290C1A05041389910B1508C059
:10DF50003401FF01FF01FF01CB13119A1408DD9872
:10DF60001B08B504132D9942081359A81B085D041A
:10DF700013D40E42201008C0A86401FFFFFF150C47
:10DF800029AB7C1A020E32671B138809642901F63B
:10DF900002FF0101FF01FF01FF01FF01FF01FF017E
:10DFA000FF01FF01111385A11408619F140885A5C5
:10DFB0001408F5AF140859811408E80EFA20281245
:10DFC000B7140869BA140889BE140841C80C1008AF
:10DFD0002C1824011C130DB3140871B41B085838F5
:10DFE00032011B19564C12621B08E514130DB514AF
:10DFF00008915F5B08885413B4DB140870D81B08C1
:10E0000098041AC0041AE8041310D91B0838041B1A
:10E01000B8D6281920137CDD1B0878081A68041A62
:10E020000C201AD4181A74201A040C1308DE1B08CA
:10E0300060201AA4141A10101A20041A54041A5C2E
:10E04000041A9C30132CDC1B0844041A5C041A7458
:10E05000041A8C041AA4041ABC041B88DA3C192480
:10E060001A842C2AAC5819041AFC041A245C1A4C81
:10E07000041A60041A40241A3C241A64081112D7A6
:10E080001B08F4041A14041A30041ADC181AB024F9
:10E090001AAC1C1AD4081AD0081AF8081AF4081A6C
:10E0A0001C041A18201AA09C1ABC041A50041A4006
:10E0B000041A44602A34E4190C1AF4841A14041A59
:10E0C000F4281A90381AA0041A94181A88041AF01E
:10E0D000042AD83C19681AD8041A28E80912041A24
:10E0E000E8F81ABC401AD4481A2C301A4C2C1A687A
:10E0F000041A84041AA00401FF01FF01FF01FF01BB
:10E10000FF01FF01FF01FF0140138DAA140861AE5A
:0CE11000140889AF420813081A021820F6
:04000005080028EDDA
:00000001FF
